:020000040800F2
:10000000702A0020FD010008756A00082D490008CB
:10001000716A000879040008218D000800000000C2
:10002000000000000000000000000000C58500087E
:10003000490D00080000000069710008C98500082A
:10004000170200081702000817020008C57E000802
:10005000170200081702000817020008170200081C
:10006000170200081702000817020008170200080C
:1000700017020008170200081702000817020008FC
:1000800017020008170200081702000817020008EC
:1000900017020008170200081702000817020008DC
:1000A0006D8600089D8600088D8600087D86000804
:1000B000AD860008BD860008E98600081702000822
:1000C00017020008170200081702000817020008AC
:1000D00017020008018D0008118D000817020008A2
:1000E00017020008170200081702000800F002F8C3
:1000F00000F074F814A696E8000CB244B344DA4554
:1001000001D100F06BF8BAE80F000FA696E83000B6
:10011000A5EB040504EB0607AAEB0704A7F101070A
:100120004FEA15154FEA3414A4F10104AC4201D38F
:1001300000F054F813F0010F18BFFB1A43F001034D
:1001400000F001F8DBE71847149C0000349C000025
:100150000A4410F8013B13F0030408BF10F8014BE8
:100160001D1108BF10F8015B641E05D010F8016B6B
:10017000641E01F8016BF9D1002D15D010F8014B68
:1001800003F00C030C2BA1EB04040ABF10F8013B95
:10019000A4EB8314A4EB032405F1010314F8016B11
:1001A0005B1E01F8016BF9D5914238BF10F8013B95
:1001B000D1D370477047000000230024002500269B
:1001C000103A28BF78C1FBD8520728BF30C148BFBA
:1001D0000B6070471FB51FBD10B510BD00F0CFF804
:1001E0001146FFF7F7FF08F0BFFE00F0EDF803B48B
:1001F000FFF7F2FF03BC00F0F5F800000948804764
:1002000009480047FEE7FEE7FEE7FEE7FEE7FEE7F8
:10021000FEE7FEE7FEE7FEE704480549054A064B10
:100220007047000069860008ED0000087024002077
:10023000702A00207026002070260020032A40F239
:10024000308010F0030C00F0158011F8013BBCF178
:10025000020F624498BF11F801CB00F8013B38BF90
:1002600011F8013BA2F1040298BF00F801CB38BF9E
:1002700000F8013B11F0030300F04F80083AC0F092
:10028000088051F8043B083A51F804CBA0E8081064
:10029000F5E7121D5CBF51F8043B40F8043BAFF397
:1002A0000080D20724BF11F8013B11F801CB48BFF1
:1002B00011F8012B24BF00F8013B00F801CB48BF27
:1002C00000F8012B70474FF0000200B5134694462A
:1002D0009646203922BFA0E80C50A0E80C50B1F19E
:1002E0002001BFF4F7AF090728BFA0E80C5048BFB2
:1002F0000CC05DF804EB890028BF40F8042B08BF50
:10030000704748BF20F8022B11F0804F18BF00F84B
:10031000012B704770477047704710B5203AC0F006
:100320000B80B1E81850A0E81850B1E81850A0E8C8
:100330001850203ABFF4F5AF5FEA027C24BFB1E861
:100340001850A0E8185044BF18C918C0BDE81040A4
:100350005FEA827C24BF51F8043B40F8043B08BFAD
:100360007047D20728BF31F8023B48BF11F8012B74
:1003700028BF20F8023B48BF00F8012B70477546A4
:1003800000F02CF8AE4605006946534620F0070001
:10039000854618B020B5FFF73FFFBDE820404FF07D
:1003A00000064FF000074FF000084FF0000BAC467E
:1003B000ACE8C009ACE8C009ACE8C009ACE8C009C9
:1003C00021F007018D46704710B50446AFF3008059
:1003D0002046BDE81040FFF70ABF00000048704704
:1003E0001802002001491820ABBEFEE726000200DB
:1003F0007047000080B584B0029000200190029800
:1004000000688068C00770B3FFE7029801688868D9
:1004100020F00100886001F0EBFA0190FFE70298FC
:1004200000688068C007E8B1FFE701F0E1FA0199D0
:10043000401A032815D3FFE7029800688068C007B8
:1004400070B1FFE70299886A40F010008862029953
:10045000C86A40F00100C86201208DF80F0006E074
:10046000FFE7DCE7FFE700208DF80F00FFE79DF8CE
:100470000F0004B080BD0000FFE7FEE780B586B046
:10048000059004910392029300200190FFE70198E8
:1004900003990968C97A884213DAFFE70198C0EB2B
:1004A000C00141F69020C2F2000010F8310080082F
:1004B000C00708B1FFE7FFE7FFE7019801300190AF
:1004C000E5E741F63820C2F20000006828B9FFE7EE
:1004D00004980078C007F0B1FFE741F63821C2F276
:1004E0000001002008600499087800F0FE00087000
:1004F00040F27820C2F2000041F2E031C2F2000185
:1005000000F040F909F044F803980068C07A0599B2
:10051000A1F86009FFE706B080BD000080B58AB091
:100520000890079106920593089820B9FFE70120EB
:100530008DF82700B7E0079820B9FFE701208DF874
:100540002700B0E0069820B9FFE701208DF82700CA
:10055000A9E0059820B9FFE701208DF82700A2E067
:1005600000208DF80F00079800F0A2F820B1FFE7F7
:1005700001208DF8270096E006990878497840EA2E
:100580000120ADF81200089806F05CFCBDF81200DE
:100590000004002809D5FFE7BDF812004042ADF87D
:1005A000120001208DF80F00FFE7069800798DF802
:1005B0001100BDF8120000098DF810009DF813001D
:1005C00000F007019DF8100040EA01108DF81000BE
:1005D0009DF81100014601911F280CD0FFE70198FA
:1005E0003F2816D0FFE701985F2820D0FFE7019849
:1005F0007F282AD037E0BDF81200C0F3C00009F010
:10060000AFF9029002984FF07C5109F03DFA029048
:1006100030E0BDF81200C0F3810009F0A1F90290AA
:1006200002984FF07A5109F02FFA029022E0BDF8BB
:100630001200C0F3420009F093F9029002984FF0C3
:10064000785109F021FA029014E0BDF8120000F090
:100650000F0009F085F9029002984FF0765109F0E9
:1006600013FA029006E005990020086001208DF839
:10067000270018E09DF9100009F072F9029909F0BD
:1006800087F802909DF80F0030B1FFE70299002033
:1006900009F0C6FA0290FFE7029805990860002069
:1006A0008DF82700FFE79DF827000AB080BD000005
:1006B00082B00090009820B9FFE701208DF8070074
:1006C0000CE000980078282804D1FFE700208DF87E
:1006D000070003E001208DF80700FFE79DF8070001
:1006E00002B0704780B586B00490039102920498DE
:1006F00020B9FFE701208DF817003FE0039820B9EB
:10070000FFE701208DF8170038E0029820B9FFE7D5
:1007100001208DF8170031E0049806F093FB04984F
:10072000039906F0A7FA0498BE2106F0F9FC002010
:100730000190FFE7019808280BDCFFE7049806F01A
:100740004FFB0299019A8854FFE70198013001900C
:10075000F0E70298082106F0C5F98DF803009DF82E
:1007600003000299097A884204D0FFE701208DF83E
:10077000170003E000208DF81700FFE79DF8170031
:1007800006B080BD80B586B004900391039820B96F
:10079000FFE701208DF8170044E003990020C8729C
:1007A000FFE70398F02106F07DFB012801D0FFE769
:1007B0000BE003980499C27A01EBC20106F012FA29
:1007C0000399C87A0130C872EBE70398C07A0290A7
:1007D000FFE702981F2818DCFFE700200190FFE7E1
:1007E000019807280CDCFFE70498029900EBC1018F
:1007F000019A00208854FFE7019801300190EFE74B
:10080000FFE7029801300290E3E70398C07A0128DD
:1008100004DBFFE700208DF8170003E002208DF8CD
:100820001700FFE79DF8170006B080BD80B584B0C3
:10083000029001918DF80320029820B9FFE7012072
:100840008DF80F005CE0019820B9FFE701208DF8DA
:100850000F0055E00198FFF72BFF20B1FFE70120C3
:100860008DF80F004CE0029806F0ECFA029801991E
:1008700006F000FA0298BE2106F052FC029806F03B
:10088000AFFA029806F0ACFA029806F0A9FA8DF8D1
:100890000200029806F0A4FA8DF80100029806F012
:1008A0009FFA8DF800009DF803008DF80000029873
:1008B00006F0C8FA0298019906F0DCF902984E2178
:1008C00006F02EFC02989DF8021006F029FC029812
:1008D0009DF8011006F024FC02989DF8001006F027
:1008E0001FFC029806F0AEFA0298019906F0C2F9D0
:1008F0000298482106F014FC00208DF80F00FFE755
:100900009DF80F0004B080BD80B582B000900098C3
:1009100020B9FFE701208DF807000EE0009806F0EF
:1009200091FA0098CC2106F0FBFB0098442106F0D8
:10093000F7FB00208DF80700FFE79DF8070002B0E5
:1009400080BD000080B584B00290029820B9FFE716
:1009500001208DF80F001AE001F04AF80190FFE73E
:10096000029806F007FA70B9FFE701F041F8019923
:10097000401A40F2EF21884204D3FFE703208DF8AC
:100980000F0004E0ECE700208DF80F00FFE79DF872
:100990000F0004B080BD000080B584B002900191CA
:1009A000029820B9FFE701208DF80F0015E00198AB
:1009B00020B9FFE701208DF80F000EE002980199A1
:1009C00008610199D1F82D20029890478DF8030015
:1009D0009DF803008DF80F00FFE79DF80F0004B0AD
:1009E00080BD000080B586B00490049820B9FFE770
:1009F00001208DF8170026E0049802F08DFF41F2E7
:100A00005062C2F2000241F2E030C2F200000290F5
:100A1000106040F27821C2F20001019151604FF460
:100A20000041818140F60001C4F20101016106F03C
:100A3000F5F801980299FFF7A5FE002818BF0120DC
:100A40008DF81700FFE79DF8170006B080BD000085
:100A500080B584B00290029820B9FFE701208DF89C
:100A60000F0031E0029800F033F88DF807009DF890
:100A7000070070B9FFE70299087840F0010008709C
:100A80000299087800F0FB00087000208DF80F0034
:100A90001AE002990020086202980078C00728B185
:100AA000FFE70299087901300871FFE70299087899
:100AB00040F0040008700299087800F0FE00087009
:100AC00002208DF80F00FFE79DF80F0004B080BDF5
:100AD00080B582B00090009820B9FFE701208DF822
:100AE000070009E000990A6952F8080B1831FFF76E
:100AF000F9FD8DF80700FFE79DF8070002B080BD03
:100B000080B584B00290029820B9FFE701208DF8EB
:100B10000F0033E0029800784008C00720B9FFE7D3
:100B200001208DF80F0029E00298FFF791FF8DF862
:100B300007009DF8070028B1FFE79DF807008DF832
:100B40000F001BE0029B1A6952F8080B03F1180111
:100B50002033FFF7E3FC8DF807009DF8070048B14C
:100B6000FFE702994879013048719DF807008DF838
:100B70000F0003E000208DF80F00FFE79DF80F0045
:100B800004B080BD80B586B00490039102920398B2
:100B900020B9FFE701208DF8170047E0049820B93D
:100BA000FFE701208DF8170040E0049803990861E1
:100BB00003990020C8618861029908684A6803990E
:100BC000CA6188610398FFF783FF8DF807009DF8DD
:100BD000070008BBFFE7049800680299039A92F89F
:100BE0002C20FFF723FE8DF807009DF8070048B979
:100BF000FFE70399087840F00200087000208DF8A4
:100C0000170013E00399087800F0FD0008709DF8C4
:100C100007008DF8170009E00399087800F0FD003F
:100C200008709DF807008DF81700FFE79DF8170082
:100C300006B080BD80B584B002900191029820B9C1
:100C4000FFE701208DF80F0015E0019820B9FFE7BC
:100C500001208DF80F000EE00298019942684B6A5E
:100C600002EBC302FFF78EFF8DF803009DF803002F
:100C70008DF80F00FFE79DF80F0004B080BD000065
:100C800080B586B004908DF80F108DF80E20049872
:100C900020B9FFE701208DF8170050E004980068A4
:100CA000FFF732FE8DF80D009DF80D0028B1FFE72B
:100CB0009DF80D008DF8170041E09DF80F00012808
:100CC0000BD1FFE704980068FFF73CFE8DF80D009C
:100CD0009DF80D008DF8170031E09DF80F000228F7
:100CE00028D1FFE7002002909DF80E0001460191F7
:100CF0001F280CD0FFE701983F280BD0FFE7019891
:100D00005F280AD0FFE701987F280AD00DE05E2017
:100D100002900BE0BC20029008E040F277100290B5
:100D200004E040F2EE20029000E0FFE7029800F0BD
:100D300095FCFFE79DF80D008DF81700FFE79DF883
:100D4000170006B080BD00007047000081B0EFF3CF
:100D5000108072B60090FFE7FEE7000080B584B017
:100D600003900291039800F5FA6041F25061C2F2DB
:100D7000000149684FF48072FFF760FA039807F0AA
:100D800069F9039890F8A4090299C0F34002087821
:100D900000F0FE00104408700398022108F01EFACB
:100DA00041F2F740C2F20000007830B9FFE7039843
:100DB00090F8A409C007E8B3FFE741F2F741C2F297
:100DC000000100200870039AB2F8A41921F0010173
:100DD000A2F8A4190190FFE7019841F25061C2F214
:100DE00000010968C97A884223DAFFE7039801996C
:100DF000009100EB4100B0F8A60908F0C9FD009988
:100E0000C1EBC10241F69021C2F2000101EBC20226
:100E100090600398019A00EB4200B0F86E0AC2EBB2
:100E2000C20201EBC2018881FFE701980130019005
:100E3000D2E7FFE7002004B080BD000085B003903A
:100E4000029100208DF807000090FFE7039890F8CA
:100E50002400012804D1FFE702208DF81300C3E02D
:100E60000399012081F82400FFE7FFE7029840681A
:100E7000062812D8FFE703980068406B029A1168B1
:100E8000526802EB8202053A1F2393409843914037
:100E9000084303990968486329E0029840680C28D0
:100EA00012D8FFE703980068006B029A1168526835
:100EB00002EB8202233A1F23934098439140084358
:100EC00003990968086311E003980068C06A029AF0
:100ED0001168526802EB8202413A1F239340984303
:100EE0009140084303990968C862FFE7FFE7029849
:100EF00000680A2812D3FFE703980068C0680299C7
:100F00000A68896802EB42021E3A0723934098431D
:100F10009140084303990968C86010E0039800688D
:100F2000006902990A68896802EB4202072393402C
:100F3000984391400843039909680861FFE70298C4
:100F40000068102805D0FFE702980068112840D1FA
:100F5000FFE70398006842F20041C4F201018842B1
:100F60002DD1FFE70398006880680002002825D48F
:100F7000FFE703980168886840F4000088600298E1
:100F80000068102819D1FFE740F20000C2F200000B
:100F900000684DF68361C4F21B31A0FB0110800C88
:100FA00000EB800040000090FFE7009820B1FFE7D1
:100FB000009801380090F8E7FFE7FFE708E00399A1
:100FC000886A40F02000886201208DF80700FFE762
:100FD000FFE7FFE70399002081F82400FFE79DF871
:100FE00007008DF81300FFE79DF8130005B0704768
:100FF00080B588B0069000208DF81700049003900B
:101000000290069820B9FFE701208DF81F00F4E058
:101010000698806830B1FFE70698007D08B1FFE7C9
:10102000FFE7FFE70698806A50B9FFE706990020BE
:10103000C862069981F82400069800F0E3F8FFE7FB
:101040000698FFF7D7F98DF817000698806AC00652
:10105000002800F1C480FFE79DF81700002840F049
:10106000BE80FFE70698806A40F0020020F48850B6
:101070000699886206994868CA691043097B40EA64
:101080004101039808430390069881680120B1F557
:10109000807F019008D0FFE7069880680138B0FA99
:1010A00080F040090190FFE701990498CA0740F4D5
:1010B0008071002A18BF084604900698007D012818
:1010C0001ED1FFE70698007B70B9FFE7069881699B
:1010D0004EF20000CFF6FF7000EB41300499084358
:1010E00040F4006004900AE00699886A40F020000D
:1010F00088620699C86A40F00100C862FFE7FFE70E
:1011000006980068406820F46940049908430699ED
:10111000096848600698006880684FF2FD71CFF654
:10112000E1710840039908430699096888600698A8
:1011300081680120B1F5807F009008D0FFE7069814
:1011400080680138B0FA80F040090090FFE700980D
:1011500000F00100002818BF4FF48070B0F5807FC8
:1011600009D1FFE7069801690020CFF6F07000EB87
:1011700001500290FFE706980068C06A20F47000F2
:101180000299084306990968C86206980068806851
:1011900040F6FE61CFF61F710840039988420CD1DA
:1011A000FFE706990020C8620698806A40F00100B7
:1011B00020F002000699886210E00698806A40F0EC
:1011C000100020F00200069988620699C86A40F073
:1011D0000100C86201208DF81700FFE708E00699BA
:1011E000886A40F01000886201208DF81700FFE740
:1011F0009DF817008DF81F00FFE79DF81F0008B04D
:1012000080BD000082B001900198006842F2004168
:10121000C4F20101884210D1FFE7FFE741F2180054
:10122000C4F20200016841F400710160006800F43A
:10123000007000900098FFE7FFE702B070470000E1
:1012400080B584B00290029820B9FFE701208DF8A4
:101250000F00E0E0029890F8200020B9FFE7029824
:1012600000F0DEF8FFE702980168086840F001002E
:10127000086000F0BDFB0190FFE70298006840683D
:10128000C007A8B9FFE700F0B3FB0199401A0B288B
:101290000DD3FFE70299486A40F400304862029992
:1012A000052081F8200001208DF80F00B3E0E4E76D
:1012B00002980168086820F00200086000F098FBBE
:1012C0000190FFE70298006840688007002815D564
:1012D000FFE700F08DFB0199401A0B280DD3FFE7C3
:1012E0000299486A40F4003048620299052081F86A
:1012F000200001208DF80F008DE0E3E70298007ECA
:10130000012807D1FFE702980168086840F08000D3
:10131000086006E002980168086820F08000086014
:10132000FFE70298407E012807D1FFE70298016895
:10133000086840F04000086006E00298016808680C
:1013400020F040000860FFE70298807E012807D166
:10135000FFE702980168086840F02000086006E096
:1013600002980168086820F020000860FFE70298F2
:10137000C07E012807D1FFE702980168086820F0C5
:101380001000086006E002980168086840F010004C
:101390000860FFE70298007F012807D1FFE7029865
:1013A0000168086840F00800086006E002980168DB
:1013B000086820F008000860FFE70298407F0128D5
:1013C00007D1FFE702980168086840F00400086050
:1013D00006E002980168086820F004000860FFE752
:1013E000029B19685A689868D3F80CC040EA0C0050
:1013F000D3F810C040EA0C005B691843013A10436F
:10140000C861029900204862029A012182F82010E6
:101410008DF80F00FFE79DF80F0004B080BD0000BD
:1014200080B58AB00990002008900790069005903A
:101430000998006846F20041C4F20001884239D19F
:10144000FFE7FFE741F21C00C4F20200016841F02F
:1014500000710160006800F0007004900498FFE7DC
:10146000FFE741F21800C4F20200016841F00401F4
:101470000160006800F0040003900398FFE74FF458
:101480000060059000200690079040F60000C4F22E
:101490000100019005A9029100F002F9019802995A
:1014A0004FF480520592022206920322089200F025
:1014B000F7F8FFE70AB080BD83B0019000208DF8F7
:1014C0000300019890F8210002280DD0FFE7019950
:1014D00004208863FFE70199002081F82000FFE7DE
:1014E00001208DF80B0021E001980168086820F0C8
:1014F0000E00086001980168086820F0010008608B
:101500000198C16B026C012090404860FFE701998F
:10151000012081F82100FFE70199002081F82000D7
:10152000FFE79DF803008DF80B00FFE79DF80B0027
:1015300003B0704780B588B0079000208DF81B007D
:10154000079890F82100022807D0FFE707990420A8
:10155000886301208DF81B0076E007980168086811
:1015600020F00E00086007980168086820F001006C
:101570000860079800680821C4F20201884203D17C
:10158000FFE70120059047E0079800681C21C4F29E
:101590000201884203D1FFE71020049039E0079848
:1015A00000683021C4F20201884204D1FFE74FF401
:1015B000807003902AE0079800684421C4F2020179
:1015C000884204D1FFE74FF4805002901BE0079857
:1015D00000685821C4F20201884204D1FFE74FF4A9
:1015E000803001900CE0079801686C22C4F202027E
:1015F0004FF08070914208BF4FF480100190FFE7D8
:1016000001980290FFE702980390FFE70398049087
:10161000FFE704980590FFE705980421C4F2020152
:1016200008600799012081F82100FFE70799002051
:1016300081F82000FFE70798406B20B1FFE707988B
:10164000416B8847FFE7FFE79DF81B0008B080BDAE
:1016500081B000900098806B01B0704780B584B075
:10166000039000F0C5F902900398019001980130B1
:1016700048B1FFE740F21220C2F200000178019861
:1016800008440190FFE7FFE700F0B2F90299401A21
:101690000199884201D2FFE7F6E704B080BD00005F
:1016A00090B00F900E9100200D900990FFE70E98DA
:1016B00000680D99C840002800F07F81FFE70D9970
:1016C000012088400C900E9800680C9908400B90FF
:1016D0000B980C99884240F06C81FFE70E984068A7
:1016E0000590002851D0FFE7059801283AD0FFE780
:1016F000059802283FD0FFE7059803285FD0FFE751
:101700000598112832D0FFE70598122838D0FFE756
:1017100005980021C1F21101884236D0FFE70598F3
:101720000021C1F2120188422FD0FFE70598002165
:10173000C1F22101884228D0FFE705980021C1F2BB
:101740002201884221D0FFE705980021C1F2310132
:1017500088421AD0FFE705980021C1F23201884281
:1017600013D02FE00E98C06809902CE00E98C06846
:101770000430099027E00E98C0680830099022E0F4
:101780000E98C0680C3009901DE00E98806818B95A
:10179000FFE70420099011E00E988068012806D127
:1017A000FFE7082009900C980F99086105E00820D0
:1017B00009900C980F994861FFE7FFE703E00020CC
:1017C000099000E0FFE70B98FF2803D8FFE70F9888
:1017D000049003E00F9804300490FFE70498089009
:1017E0000B98FF2804D8FFE70D988000039006E0CF
:1017F0000D996FF01F0000EB81000390FFE7039845
:10180000079008980068079A0F219140884309992A
:1018100091400843089908600E98C079C0060028D6
:1018200040F1C680FFE7FFE741F21800C4F2020072
:10183000016841F001010160006800F001000690BC
:101840000698FFE70D9820F003000821C4F201017B
:1018500040580A900D9800F0030081000F2000FA14
:1018600001F10A9888430A900F9840F60001C4F2EB
:101870000101884203D1FFE70020029026E00F9883
:1018800040F60041C4F20101884203D1FFE7012084
:10189000019018E00F9841F20001C4F20101884262
:1018A00003D1FFE7022000900AE00F9941F20042C5
:1018B000C4F201020420914208BF03200090FFE718
:1018C00000980190FFE701980290FFE702980D99B8
:1018D00001F00301890000FA01F10A9808430A9017
:1018E0000A980D9921F003010822C4F201028850E0
:1018F0000E988079C006002809D5FFE70B9A40F2C0
:101900000841C4F2010108681043086008E00B9A1E
:1019100040F20841C4F20101086890430860FFE703
:101920000E9880798006002809D5FFE70B9A40F2CF
:101930000C41C4F2010108681043086008E00B9AEA
:1019400040F20C41C4F20101086890430860FFE7CF
:101950000E9880798007002809D5FFE70B9A40F29E
:101960000441C4F2010108681043086008E00B9AC2
:1019700040F20441C4F20101086890430860FFE7A7
:101980000E988079C00748B1FFE70B9A40F20041FA
:10199000C4F2010108681043086008E00B9A40F2A5
:1019A0000041C4F20101086890430860FFE7FFE7C7
:1019B000FFE70D9801300D9079E610B070470000F8
:1019C00082B00190ADF802108DF801209DF8010061
:1019D00028B1FFE7BDF802000199086105E0BDF8F4
:1019E0000200000401990861FFE702B0704700009F
:1019F00042F26C40C2F200000068704780B58EB0C1
:101A00000C900C9820B9FFE701208DF8370043E1D6
:101A10000C9890F83D0040B9FFE70C99002081F840
:101A20003C000C9800F03CF9FFE70C99242081F869
:101A30003D000C980168086820F0010008600C98CF
:101A40000168086840F4004008600C980168086864
:101A500020F40040086000F081FD0A900C98406876
:101A600048F2A061C0F2010188420BD8FFE70A9951
:101A700048F28042C0F21E020020914238BF01208D
:101A800009900AE00A9940F60012C0F23D020020D7
:101A9000914238BF01200990FFE70998012804D13D
:101AA000FFE701208DF83700F6E00A984DF68361D4
:101AB000C4F21B31A0FB0110800C0B900C98006845
:101AC000406820F03F000B9908430C990968486072
:101AD0000C980068006A20F03F0008900C9840685D
:101AE00048F2A061C0F20101884204D8FFE70B98D8
:101AF000013007900EE00B984FF49671484344F67E
:101B0000D351C1F26201A0FB0101012000EB911051
:101B10000790FFE70898079908430C99096808623D
:101B20000C980068C0694CF6FF71884306900C98C9
:101B3000406848F2A061C0F2010188421FD8FFE767
:101B40000A9801380C9949684900B0FBF1F001305E
:101B50006FF31F30032803D8FFE7042005900BE044
:101B60000A9801380C9949684900B0FBF1F001303E
:101B70006FF31F300590FFE7059804904CE00C9838
:101B8000806868B9FFE70A9801380C99496801EB49
:101B90004101B0FBF1F001306FF31F3003900DE015
:101BA0000A9801380C99496819225143B0FBF1F0A9
:101BB0000130042161F31F300390FFE70398000513
:101BC00018B9FFE70120029023E00C98806868B9FB
:101BD000FFE70A9801380C99496801EB4101B0FB15
:101BE000F1F001306FF31F3001900DE00A980138D9
:101BF0000C99496819225143B0FBF1F001300421DE
:101C000061F31F300190FFE7019840F4004002901B
:101C1000FFE702980490FFE70698049908430C999F
:101C20000968C8610C980068006820F0C0000C9B2F
:101C30001968DA691B6A1A43104308600C98006837
:101C4000806848F2FF3188430C9A1168D3681269A2
:101C50001A43104388600C980068C06820F0FF00A9
:101C60000C9B19685A699B691A431043C8600C9809
:101C70000168086840F0010008600C9900200864C1
:101C80000C9A202182F83D100C9908630C9981F878
:101C90003E008DF83700FFE79DF837000EB080BD9D
:101CA00080B588B0079000200690059004900390BE
:101CB0000798006845F20041C4F20001884240D113
:101CC000FFE7FFE741F21800C4F20200016841F0AB
:101CD00008010160006800F0080002900298FFE728
:101CE0004FF44070039012200490002005900320D0
:101CF000069040F60040C4F2010003A9FFF7D0FCB3
:101D0000FFE70421C4F2010108680190019840F046
:101D1000E0600190019840F0020001900198086095
:101D2000FFE7FFE741F21C00C4F20200016841F442
:101D300000110160006800F4001000900098FFE7B7
:101D4000FFE708B080BD000040F21220C2F20000A0
:101D5000027842F26C41C2F2000108681044086047
:101D60007047000080B542F20001C4F20201086829
:101D700040F010000860032000F0D6F80F2000F0BB
:101D800005F800F07BF8002080BD000080B58CB025
:101D90000B900020049003908DF80700FFE741F2BC
:101DA0001C00C4F20200016841F0020101600068F9
:101DB00000F0020000900098FFE706A802A900F0DA
:101DC0009DFB09980490049820B9FFE700F0C6FB3A
:101DD000059004E000F0C2FB40000590FFE7059885
:101DE0004DF68361C4F21B31A0FB01014FF0FF30BF
:101DF00000EB9140039041F61810C2F2000040F24F
:101E00000041C4F20001016040F2E731C160039972
:101E10004160002101618160816101F0A9FC8DF8C0
:101E200007009DF8070028BBFFE741F61810C2F233
:101E3000000001F0C3FD8DF807009DF80700C0B950
:101E4000FFE71D2000F04CF80B980F280CD8FFE797
:101E50000B991D20002200F04DF80B9840F2142140
:101E6000C2F20001086003E001208DF80700FFE7DF
:101E7000FFE7FFE79DF807000CB080BD83B0FFE7E8
:101E800041F21800C4F20200016841F00101016052
:101E9000006800F0010002900298FFE7FFE741F2BE
:101EA0001C00C4F20200016841F08051016000682A
:101EB00000F0805001900198FFE7FFE70421C4F291
:101EC000010108680090009820F0E0600090009800
:101ED00040F00070009000980860FFE703B0704782
:101EE00080B582B08DF807009DF9070006F01AFF53
:101EF00002B080BD80B586B08DF8170004910392C2
:101F00000020029006F026FF02909DF91700019034
:101F100002980499039A04F0AFFD0146019806F077
:101F200021FF06B080BD000080B582B0019001980D
:101F300006F03AFF02B080BD2021C4F20E2101203C
:101F40000860704780B588B0079000200690059023
:101F500004900390029007980190012866D0FFE753
:101F60000198022800F0A580FFE70198102840F0B2
:101F7000B080FFE741F20400C4F202000068039061
:101F800041F20000C4F202000068C00100284CD5F4
:101F9000FFE70398C0F3834149F62250C0F60000E2
:101FA000405C04909DF80E00C007F0B1FFE741F2DD
:101FB0000400C4F202000068C0F3404149F6325008
:101FC000C0F60000405C06909DF80E00C00758B1B6
:101FD000FFE7069941F20020C0F27A00B0FBF1F071
:101FE000049948430590FFE707E0049840F6001184
:101FF000C0F23D0148430590FFE741F20400C4F2FE
:10200000020000684002002803D5FFE7059802900F
:102010000AE0059840004AF6AB21CAF6AA21A0FBC7
:10202000011040080290FFE7FFE753E041F2200073
:10203000C4F2020000680390039800F44070B0F509
:10204000807F0AD1FFE79DF80C008007002804D5A7
:10205000FFE74FF4004002902AE0039800F440703C
:10206000B0F5007F0DD1FFE741F22400C4F2020079
:1020700000688007002804D5FFE749F64040029039
:1020800015E0039800F44070B0F5407F0DD1FFE7F4
:1020900041F20000C4F2020000688003002804D569
:1020A000FFE74FF22440029000E0FFE7FFE7FFE781
:1020B00010E000F065FA41F20401C4F2020109687F
:1020C00001F44042022101EB5231B0FBF1F00290E9
:1020D00000E0FFE7029808B080BD000080B586B040
:1020E000049000200390029004980078C007002814
:1020F00000F0AC80FFE700208DF8070041F21C00E3
:10210000C4F202000068C000002813D4FFE7FFE714
:1021100041F21C00C4F20200016841F080510160EC
:10212000006800F0805000900098FFE701208DF8D3
:102130000700FFE747F20000C4F200000068C00596
:10214000002822D4FFE747F20001C4F2000108682A
:1021500040F480700860FFF74BFC0390FFE747F204
:102160000000C4F200000068C00500280CD4FFE79E
:10217000FFF73EFC0399401A652804D3FFE70320CC
:102180008DF817008AE0EAE7FFE741F22000C4F289
:102190000200006800F4407002900298E0B3FFE78C
:1021A00002980499496801F44071884234D0FFE7ED
:1021B00041F22001C4F20201086820F4407002904C
:1021C00040F24042C4F24222012010600020106020
:1021D000029808609DF80800C007E0B1FFE7FFF72C
:1021E00007FC0390FFE741F22000C4F20200006800
:1021F000800700280ED4FFE7FFF7FAFB0399401A87
:1022000041F28931884204D3FFE703208DF817009B
:1022100044E0E8E7FFE7FFE741F22001C4F20201F2
:10222000086820F44070049A5268104308609DF8D2
:102230000700012809D1FFE741F21C01C4F20201A5
:10224000086820F080500860FFE7FFE704980078F6
:10225000800700280CD5FFE741F20401C4F2020117
:10226000086820F44040049A926810430860FFE731
:1022700004980078C00600280CD5FFE741F204015D
:10228000C4F20201086820F48000049AD268104366
:102290000860FFE700208DF81700FFE79DF81700A2
:1022A00006B080BD80B584B002900191029820B93B
:1022B000FFE701208DF80F001BE1019842F20001B9
:1022C000C4F20201096801F00701884216D9FFE74C
:1022D00042F20000C4F20200016821F00701019AF5
:1022E00011430160006800F007000199884204D0A2
:1022F000FFE701208DF80F00FBE0FFE70298007870
:10230000800700282AD5FFE70298007840070028B8
:1023100009D5FFE741F20401C4F20201086840F464
:10232000E0600860FFE7029800780007002809D500
:10233000FFE741F20401C4F20201086840F4605072
:102340000860FFE741F20401C4F20201086820F0CE
:10235000F000029A926810430860FFE70298007844
:10236000C007002860D0FFE70298406801280ED11E
:10237000FFE741F20000C4F2020000688003002879
:1023800004D4FFE701208DF80F00B2E021E00298AD
:10239000406802280ED1FFE741F20000C4F20200BB
:1023A00000688001002804D4FFE701208DF80F00A9
:1023B0009FE00DE041F20000C4F2020000688007D7
:1023C000002804D4FFE701208DF80F0091E0FFE71B
:1023D000FFE741F20401C4F20201086820F00300A3
:1023E000029A526810430860FFF702FB0090FFE773
:1023F00041F20400C4F20200006800F00C000299EF
:102400004968B0EB810F0ED0FFE7FFF7F1FA0099B2
:10241000401A41F28931884204D3FFE703208DF846
:102420000F0066E0E4E7FFE7019842F20001C4F222
:102430000201096801F00701884216D2FFE742F263
:102440000000C4F20200016821F00701019A114363
:102450000160006800F007000199884204D0FFE79E
:1024600001208DF80F0044E0FFE702980078400754
:1024700000280CD5FFE741F20401C4F2020108680C
:1024800020F4E060029AD26810430860FFE70298E7
:102490000078000700280DD5FFE741F20401C4F2DF
:1024A0000201086820F46050029A126940EAC200F2
:1024B0000860FFE700F076F841F20401C4F202017F
:1024C0000968C9B20A0949F60A51C0F60001895CD7
:1024D000C84040F20001C2F20001086040F214203E
:1024E000C2F200000068FFF751FC00208DF80F00D9
:1024F000FFE79DF80F0004B080BD000082B001909E
:10250000009101990F20086041F20400C4F202001A
:10251000016801F00301019A5160016801F0F001C6
:10252000019A9160016801F4E061019AD16000684C
:1025300000F46050C0080199086142F20000C4F242
:102540000200006800F007000099086002B07047C0
:1025500040F20000C2F200000068704780B5FFF74B
:10256000F7FF41F20401C4F202010968C1F302223B
:1025700049F61A51C0F60001895CC84080BD0000D0
:1025800080B5FFF7E5FF41F20401C4F202010968DA
:10259000C1F3C22249F61A51C0F60001895CC84055
:1025A00080BD000086B0002005900490039002904A
:1025B000019041F20400C4F2020000680590059801
:1025C00000F00C000146009100283FD0FFE7009882
:1025D000042804D0FFE70098082806D037E041F22D
:1025E0000020C0F27A00019037E00598C0F38341E3
:1025F00049F63450C0F60000405C02909DF8160089
:10260000C007C0B1FFE741F20400C4F20200006855
:10261000C0F3404149F64450C0F60000405C0490CD
:10262000029841F20021C0F27A0148430499B0FBBC
:10263000F1F0039007E0029840F60011C0F23D016E
:1026400048430390FFE70398019006E0FFE741F25B
:102650000020C0F27A000190FFE7019806B07047B1
:1026600080B586B00490049820B9FFE701208DF86A
:1026700017002EE304980078C007002800F0AE8011
:10268000FFE741F20400C4F20200006800F00C0011
:10269000042813D0FFE741F20400C4F202000068EE
:1026A00000F00C0008281BD1FFE741F20400C4F23F
:1026B00002000068C003002812D5FFE741F20000C5
:1026C000C4F2020000688003002808D5FFE70498E0
:1026D000406820B9FFE701208DF81700F9E27CE09F
:1026E000FFE704984068B0F5803F09D1FFE741F269
:1026F0000001C4F20201086840F48030086032E052
:102700000498406868B9FFE741F20001C4F2020191
:10271000086820F480300860086820F48020086091
:1027200020E004984068B0F5A02F0DD1FFE741F2FA
:102730000001C4F20201086840F4802008600868C3
:1027400040F4803008600CE041F20001C4F2020164
:10275000086820F480300860086820F48020086051
:10276000FFE7FFE7FFE7FFE704984068D0B1FFE726
:10277000FFF73EF90390FFE741F20000C4F20200C8
:102780000068800300280CD4FFE7FFF731F90399B4
:10279000401A652804D3FFE703208DF8170098E25C
:1027A000EAE719E0FFF724F90390FFE741F20000A0
:1027B000C4F202000068800300280CD5FFE7FFF791
:1027C00017F90399401A652804D3FFE703208DF811
:1027D00017007EE2EAE7FFE7FFE7FFE704980078EB
:1027E0008007002840F18D80FFE741F20400C4F229
:1027F0000200006810F00C0F13D0FFE741F2040054
:10280000C4F20200006800F00C00082829D1FFE79C
:1028100041F20400C4F202000068C003002820D482
:10282000FFE741F20000C4F20200006880070028C0
:1028300009D5FFE704980069012804D0FFE70120CB
:102840008DF8170045E241F20001C4F20201086868
:1028500020F0F800049A526940EAC2000860FFE7DD
:102860004EE00498006958B3FFE70021C4F242210A
:1028700001200860FFF7BCF80390FFE741F2000079
:10288000C4F202000068800700280CD4FFE7FFF7BD
:10289000AFF80399401A032804D3FFE703208DF80B
:1028A000170016E2EAE741F20001C4F202010868EB
:1028B00020F0F800049A526940EAC20008601EE065
:1028C0000021C4F2422100200860FFF791F8039034
:1028D000FFE741F20000C4F2020000688007002810
:1028E0000CD5FFE7FFF784F80399401A032804D3B7
:1028F000FFE703208DF81700EBE1EAE7FFE7FFE7CA
:10290000FFE7049800780007002848D5FFE70498FF
:10291000806918B3FFE740F28041C4F242210120F0
:102920000860FFF765F80390FFE741F22400C4F266
:1029300002000068800700280CD4FFE7FFF758F872
:102940000399401A032804D3FFE703208DF81700EA
:10295000BFE1EAE7012004F009FC1FE040F28041FA
:10296000C4F2422100200860FFF742F80390FFE71D
:1029700041F22400C4F202000068800700280CD550
:10298000FFE7FFF735F80399401A032804D3FFE760
:1029900003208DF817009CE1EAE7FFE7FFE70498C2
:1029A00000784007002840F1D880FFE700208DF82C
:1029B000070041F21C00C4F202000068C0000028B9
:1029C00013D4FFE7FFE741F21C00C4F202000168E4
:1029D00041F080510160006800F080500090009844
:1029E000FFE701208DF80700FFE747F20000C4F27F
:1029F00000000068C005002822D4FFE747F200016C
:102A0000C4F20001086840F480700860FEF7F0FF2F
:102A10000390FFE747F20000C4F200000068C00521
:102A200000280CD4FFE7FEF7E3FF0399401A65285E
:102A300004D3FFE703208DF817004AE1EAE7FFE738
:102A4000FFE70498C068012809D1FFE741F220019F
:102A5000C4F20201086840F00100086031E0049807
:102A6000C06868B9FFE741F22001C4F202010868BA
:102A700020F001000860086820F0040008601FE0F2
:102A80000498C06805280DD1FFE741F22001C4F287
:102A90000201086840F004000860086840F0010086
:102AA00008600CE041F22001C4F20201086820F045
:102AB00001000860086820F004000860FFE7FFE7F5
:102AC000FFE7FFE70498C068E0B1FFE7FEF790FF7B
:102AD0000390FFE741F22000C4F202000068800783
:102AE00000280ED4FFE7FEF783FF0399401A41F256
:102AF0008931884204D3FFE703208DF81700E8E00E
:102B0000E8E71BE0FEF774FF0390FFE741F22000C7
:102B1000C4F202000068800700280ED5FFE7FEF728
:102B200067FF0399401A41F28931884204D3FFE7D5
:102B300003208DF81700CCE0E8E7FFE79DF80700D9
:102B4000012809D1FFE741F21C01C4F20201086823
:102B500020F080500860FFE7FFE70498C069002874
:102B600000F0B380FFE741F20400C4F20200006805
:102B700000F00C00082800F08280FFE70498C0698C
:102B800002285CD1FFE76021C4F2422100200860E6
:102B9000FEF72EFF0390FFE741F20000C4F20200AF
:102BA0000068800100280CD5FFE7FEF721FF03999C
:102BB000401A032804D3FFE703208DF8170088E0AC
:102BC000EAE70498006AB0F5803F0CD1FFE741F2D4
:102BD0000401C4F20201086820F40030049A9268EB
:102BE00010430860FFE741F20401C4F202010868E3
:102BF00020F47410049B1A6A5B6A1A43104308603D
:102C00006021C4F2422101200860FEF7F1FE03902A
:102C1000FFE741F20000C4F20200006880010028D2
:102C20000CD4FFE7FEF7E4FE0399401A032804D30F
:102C3000FFE703208DF817004BE0EAE71EE0602174
:102C4000C4F2422100200860FEF7D2FE0390FFE7A5
:102C500041F20000C4F202000068800100280CD597
:102C6000FFE7FEF7C5FE0399401A032804D3FFE7E8
:102C700003208DF817002CE0EAE7FFE724E0049832
:102C8000C069012804D1FFE701208DF8170020E07A
:102C900041F20400C4F2020000680290029800F4BD
:102CA00080300499096A884208D1FFE7029800F44D
:102CB00070100499496A884204D0FFE701208DF81A
:102CC000170006E0FFE7FFE7FFE700208DF8170099
:102CD000FFE79DF8170006B080BD000084B00390A8
:102CE000029100200190009046F60040C4F20000DE
:102CF00001900299019800EB810001900198006811
:102D000080B20090009804B07047000084B0039037
:102D1000029101920020009046F60040C4F20000AB
:102D200000900299009800EB81000090BDF804002B
:102D30000099086004B0704781B0009001B07047FE
:102D400081B0009001B0704780B582B001900198C9
:102D500000680068C00718B1FFE7012018B936E025
:102D60000120A0BBFFE7019800684068C00718B1C8
:102D7000FFE7012018B929E0012038BBFFE70198DF
:102D8000006840684007002803D5FFE7012018B914
:102D90000EE0012060B9FFE70198FFF7D1FF01982D
:102DA00001686FF00400486001990420487406E04F
:102DB0000198FFF7C1FF019901204874FFE70198CE
:102DC0000168486820F001004860FFE7FFE702B0B3
:102DD00080BD000080B586B004900391029200206F
:102DE0008DF80600ADF80400049818B1FFE70398C9
:102DF00020B9FFE701208DF8170034E0049801A9FD
:102E0000002200F035F820B1FFE701208DF817000F
:102E100029E00498007B039908700498C07B03990B
:102E2000C8700498407B039948700498807B03998C
:102E30008870029898B1FFE70398C07804F0F0FD1D
:102E40000399C8700398407804F0EAFD039948702C
:102E50000398807804F0E4FD03998870FFE7002070
:102E60008DF81700FFE79DF8170006B080BD000041
:102E700080B588B0069005910492002003900290DE
:102E800001900090069818B1FFE7059820B9FFE778
:102E900001208DF81F00BDE00698006840684007DB
:102EA000002803D5FFE7012018B906E0012020B96A
:102EB000FFE701208DF81F00ACE0069805F0B6F999
:102EC000039003994BF2C530C9F2A210A1FB002177
:102ED000C90A0091039BA3FB0021C90A4FF4616258
:102EE00001FB123344F24541C0F24441A3FB01C34C
:102EF000DDF814C08CF80130039BA3FB00C0C00AAE
:102F000000FB1230A0FB0121C1EB0111A0EB8100FD
:102F100005998870009818285ED3FFE700984AF654
:102F2000AB21CAF6AA21A0FB01200009019000985C
:102F3000A0FB0121090901EB4101A0EBC1000599AA
:102F40000870069805F02EF902900298013050B1F1
:102F5000FFE702980399884205D9FFE70399029891
:102F6000401A029003E04FF0FF300290FFE7019813
:102F700040F2A32141430398A0EBC11003900698AF
:102F8000039905F0F7FA20B1FFE701208DF81F0043
:102F900040E00298013078B1FFE7039902980844B5
:102FA00002900698029905F08BFA20B1FFE7012004
:102FB0008DF81F002EE00AE00698029905F080FACD
:102FC00020B1FFE701208DF81F0023E0FFE70698FE
:102FD000019904F033FE03E0009805990870FFE7BB
:102FE000049898B1FFE70598007804F019FD059959
:102FF00008700598407804F013FD0599487005980D
:10300000807804F00DFD05998870FFE700208DF8A9
:103010001F00FFE79DF81F0008B080BD80B584B099
:10302000029000200190029820B9FFE701208DF85E
:103030000F0084E00298407C38B9FFE70299002035
:103040000874029800F080F8FFE7029902204874A3
:10305000029800F00BFA38B1FFE702990420487497
:1030600001208DF80F006AE0029804F0D3FE38B119
:10307000FFE702990420487401208DF80F005EE0FC
:1030800002980168486820F007004860029880684C
:1030900048B1FFE746F63041C4F20001086820F06D
:1030A00001000860FFE746F62C41C4F20001086801
:1030B00020F46070029A9268104308600298406899
:1030C000013020B1FFE702984068019012E0012032
:1030D000FEF738FF0190019838B9FFE70299042004
:1030E000487401208DF80F0029E001980138019003
:1030F000FFE7FFE7BDF8060000F00F00029909683E
:103100008860BDF8040002990968C860029804F05C
:10311000ADFE38B1FFE702990420487401208DF814
:103120000F000CE002990020C873029A012151732C
:10313000029A9173029A51748DF80F00FFE79DF87F
:103140000F0004B080BD000080B584B003900398E8
:10315000006842F60001C4F20001884221D1FFE775
:10316000FEF7EAFEFFE741F21C00C4F2020001682C
:1031700041F000610160006800F000600290029878
:10318000FFE740F23C41C4F24221012008600320E5
:10319000019000221146FEF7ADFE0198FEF7A0FE59
:1031A000FFE704B080BD000080B588B006900591AF
:1031B00004920020039002900190069818B1FFE756
:1031C000059820B9FFE701208DF81F00A7E0FFE771
:1031D0000698007C012804D1FFE702208DF81F002B
:1031E0009DE0069901200874FFE7FFE70699022099
:1031F0004874049868B9FFE70598C0780699C873C1
:1032000005984078069948730598807806998873E0
:1032100012E00598C07804F0EDFB0699C873059894
:10322000407804F0E7FB069948730598807804F02D
:10323000E1FB06998873FFE70698417B827BC07BA0
:1032400005F0CEF8069908730698007B059908707A
:10325000069804F0EBFF039003984BF2C531C9F2D6
:10326000A211A0FB0110C00A0190019819284AD3AD
:10327000FFE701984AF6AB21CAF6AA21A0FB01108C
:10328000000940F2A32141430398A0EBC110039031
:103290000698039905F06EF960B1FFE706990420DE
:1032A0004874FFE7069900200874FFE701208DF8B5
:1032B0001F0034E0069804F075FF02900298013078
:1032C00000B3FFE70298039988421AD2FFE70298F9
:1032D00045F28011C0F2010108440290069802995B
:1032E00005F0EEF860B1FFE7069904204874FFE7A7
:1032F000069900200874FFE701208DF81F000EE0FA
:10330000FFE7FFE7FFE7069901204874FFE706990A
:1033100000200874FFE700208DF81F00FFE79DF8EC
:103320001F0008B080BD000080B588B006900591F0
:103330000492002003900290069818B1FFE70598C8
:1033400020B9FFE701208DF81F008AE0FFE706980B
:10335000007C012804D1FFE702208DF81F0080E0E7
:10336000069901200874FFE7FFE7069902204874D8
:10337000049870B9FFE7059908784A7889784FF47E
:1033800061635843C2EB021200EB820008440390D1
:103390001BE00598007804F02DFB4FF46161484371
:1033A00000900598407804F025FB01460098C1EB99
:1033B000011100EB810001900598807804F01AFB60
:1033C0000146019808440390FFE70698039905F029
:1033D000D1F860B1FFE7069904204874FFE7069929
:1033E00000200874FFE701208DF81F0039E00698DF
:1033F0000168486820F005004860069804F0D2FE95
:1034000002900298013000B3FFE7029803998842C6
:103410001AD2FFE7029845F28011C0F20101084478
:1034200002900698029905F04BF860B1FFE7069903
:1034300004204874FFE7069900200874FFE7012084
:103440008DF81F000DE0FFE7FFE7069901204874A3
:10345000FFE7069900200874FFE700208DF81F00A1
:10346000FFE79DF81F0008B080BD000080B584B064
:10347000029000200190029820B9FFE701208DF80A
:103480000F0021E002980168486820F008004860B9
:10349000FEF7AEFA0190FFE7029800684068000767
:1034A00000280DD4FFE7FEF7A3FA0199401AB0F502
:1034B0007A7F04D9FFE703208DF80F0004E0EBE7E3
:1034C00000208DF80F00FFE79DF80F0004B080BDCD
:1034D00080B584B00290029820B9FFE701208DF8F2
:1034E0000F006EE00298406A60B9FFE702984068FA
:1034F000B0F5827F01D1FFE703E002990020C861A7
:10350000FFE705E002990020086102994861FFE7A2
:10351000029900208862029890F8510040B9FFE7B4
:103520000299002081F85000029800F04FF8FFE760
:103530000299022081F8510002980168086820F081
:1035400040000860029A019211685068D2F808C0E1
:10355000D36800F482700CF4044C604403F40063FC
:103560001844136903F002031844536903F001037C
:103570001844936903F400731844D36903F03803C3
:103580001844136A03F080031843926A02F400524D
:1035900010430860029801688269042000EA124022
:1035A000486002980168C86920F40060C861029907
:1035B00000204865029A012182F851108DF80F0011
:1035C000FFE79DF80F0004B080BD000080B58AB011
:1035D00009900020089007900690059009980068CF
:1035E00043F20001C4F20101884248D1FFE7FFE73E
:1035F00041F21800C4F20200016841F480510160F8
:10360000006800F4805004900498FFE7FFE741F25F
:103610001800C4F20200016841F00801016000686E
:1036200000F0080003900398FFE72820059002208F
:1036300006900320089040F60040C4F2010000907C
:1036400005A90191FEF72CF8009801991022059226
:10365000002206920792FEF723F8FFE70421C4F246
:10366000010108680290029840F0E0600290029820
:1036700040F00100029002980860FFE7FFE70AB0FF
:1036800080BD000081B0009001B0704781B0009013
:1036900001B0704785B003900291FFE7039890F85E
:1036A0003C00012804D1FFE702208DF813005BE005
:1036B0000399012081F83C00FFE7FFE7039902200E
:1036C00081F83D0003980068406801900398006805
:1036D00080680090019820F07000019002980168C5
:1036E000019808430190019803990968486003987C
:1036F000006842F60041C4F20101884218D0FFE799
:1037000003980068B0F1804F12D0FFE7039800687B
:1037100040F20041C4F20001884209D0FFE703985B
:10372000006840F60001C4F2000188420ED1FFE7B4
:10373000009820F0800000900298416800980843AB
:1037400000900098039909688860FFE703990120B9
:1037500081F83D00FFE70399002081F83C00FFE776
:1037600000208DF81300FFE79DF8130005B07047A7
:1037700080B582B00090009820B9FFE701208DF855
:1037800007003FE0009890F83D0040B9FFE700993E
:10379000002081F83C00009800F038F8FFE700991D
:1037A000022081F83D00009951F8040B04F0A4FFB9
:1037B0000099012081F84600FFE70099012081F877
:1037C0003E00009981F83F00009981F8400000997F
:1037D00081F84100FFE7FFE70099012081F84200EE
:1037E000009981F84300009981F84400009981F81C
:1037F0004500FFE70099012081F83D0000208DF889
:103800000700FFE79DF8070002B080BD80B58CB0CF
:103810000B900B98006842F60041C4F20101884207
:1038200035D1FFE7FFE741F21800C4F2020001685A
:1038300041F400610160006800F400600A900A9899
:10384000FFE718200390002206921146FEF752FB74
:103850000398FEF745FB069A192004901146FEF7DF
:1038600049FB0498FEF73CFB069A1A200590114686
:10387000FEF740FB0598FEF733FB069A1B200790E6
:103880001146FEF737FB0798FEF72AFB42E00B983C
:103890000068B0F1804F19D1FFE7FFE741F21C004B
:1038A000C4F20200016841F001010160006800F00B
:1038B000010009900998FFE71C20029000221146A0
:1038C000FEF718FB0298FEF70BFB22E00B9800684E
:1038D00040F60001C4F20001884219D1FFE7FFE77A
:1038E00041F21C00C4F20200016841F004010160D1
:1038F000006800F0040008900898FFE71E2001907F
:1039000000221146FEF7F6FA0198FEF7E9FAFFE702
:10391000FFE7FFE70CB080BD83B00190019890F8FD
:103920003D00012804D0FFE701208DF80B0041E0A5
:103930000199022081F83D000198006842F600419B
:10394000C4F20101884218D0FFE701980068B0F185
:10395000804F12D0FFE70198006840F20041C4F2A6
:103960000001884209D0FFE70198006840F6000195
:10397000C4F20001884212D1FFE701980068806814
:1039800000F0070000900098062807D0FFE7019894
:103990000168086840F001000860FFE706E0019850
:1039A0000168086840F001000860FFE700208DF81A
:1039B0000B00FFE79DF80B0003B0704783B0019048
:1039C000019890F83D00012804D0FFE701208DF810
:1039D0000B0047E00199022081F83D000198016841
:1039E000C86840F00100C8600198006842F60041D4
:1039F000C4F20101884218D0FFE701980068B0F1D5
:103A0000804F12D0FFE70198006840F20041C4F2F5
:103A10000001884209D0FFE70198006840F60001E4
:103A2000C4F20001884212D1FFE701980068806863
:103A300000F0070000900098062807D0FFE70198E3
:103A40000168086840F001000860FFE706E001989F
:103A50000168086840F001000860FFE700208DF869
:103A60000B00FFE79DF80B0003B0704781B000909A
:103A700000980168C86820F00100C860FFE700985E
:103A80000068006A41F21111084210D1FFE7009866
:103A90000068006A40F24441084207D1FFE70098FD
:103AA0000168086820F001000860FFE7FFE7FFE712
:103AB0000099012081F83D00002001B0704700000E
:103AC00080B586B00490039100208DF80B00FFE7CD
:103AD000049890F83C00012804D1FFE702208DF8FB
:103AE0001700ABE00499012081F83C00FFE7FFE7F5
:103AF0000499022081F83D000498006880680190D4
:103B0000019820F077000190019820F47F40019007
:103B1000019804990968886003980068009000285B
:103B200072D0FFE7009810286ED0FFE70098202899
:103B30006AD0FFE70098302866D0FFE70098402859
:103B400055D0FFE70098502837D0FFE7009860284D
:103B500040D0FFE7009870280BD0FFE70098B0F541
:103B6000805F05D0FFE70098B0F5005F16D052E007
:103B700055E004980068039B5A689968DB6804F074
:103B80003FFE0498006880680190019840F077003B
:103B90000190019804990968886040E004980068E1
:103BA000039B5A689968DB6804F02AFE0498016850
:103BB000886840F48040886031E004980068039A87
:103BC0005168D26804F04CFE04980068502104F05B
:103BD00031FE24E004980068039A5168D26804F02A
:103BE00067FE04980068602104F024FE17E0049842
:103BF0000068039A5168D26804F032FE04980068A5
:103C0000402104F017FE0AE004980068039909684F
:103C100004F010FE03E001208DF80B00FFE704998B
:103C2000012081F83D00FFE70499002081F83C0065
:103C3000FFE79DF80B008DF81700FFE79DF81700D0
:103C400006B080BD81B0009001B0704780B584B0EF
:103C5000039003980068C0680290039800680069A8
:103C600001909DF804008007002824D5FFE79DF807
:103C70000800800700281DD5FFE7039801686FF052
:103C800002000861039901200877039800688069A1
:103C9000800720B1FFE70398FFF7D4FF06E0039801
:103CA00000F0E2F8039800F0E3F8FFE70399002042
:103CB0000877FFE7FFE79DF804004007002825D5B7
:103CC000FFE79DF80800400700281ED5FFE703988E
:103CD00001686FF0040008610399022008770398D7
:103CE0000068806910F4407F04D0FFE70398FFF775
:103CF000A9FF06E0039800F0B7F8039800F0B8F8C1
:103D0000FFE7039900200877FFE7FFE79DF804002D
:103D10000007002824D5FFE79DF8080000070028C9
:103D20001DD5FFE7039801686FF00800086103994B
:103D30000420087703980068C069800720B1FFE776
:103D40000398FFF77FFF06E0039800F08DF80398D3
:103D500000F08EF8FFE7039900200877FFE7FFE700
:103D60009DF80400C006002825D5FFE79DF808004F
:103D7000C00600281ED5FFE7039801686FF0100009
:103D8000086103990820087703980068C06910F457
:103D9000407F04D0FFE70398FFF754FF06E0039845
:103DA00000F062F8039800F063F8FFE70399002041
:103DB0000877FFE7FFE79DF80400C00778B1FFE749
:103DC0009DF80800C00748B1FFE7039801686FF04D
:103DD00001000861039800F04FF8FFE7FFE79DF846
:103DE00004000006002810D5FFE79DF80800000633
:103DF000002809D5FFE7039801686FF0800008618B
:103E00000398FFF73FFCFFE7FFE79DF8040040063B
:103E1000002810D5FFE79DF808004006002809D5C6
:103E2000FFE7039801686FF040000861039800F015
:103E300035F8FFE7FFE79DF804008006002810D55D
:103E4000FFE79DF808008006002809D5FFE70398E2
:103E500001686FF0200008610398FFF717FCFFE787
:103E6000FFE704B080BD000081B0009001B0704752
:103E700081B0009001B0704780B582B00190019888
:103E8000006840F20041C4F20001884203D1FFE71C
:103E9000FDF75AFFFFE702B080BD000081B000903F
:103EA00001B0704782B00190ADF8021002B07047C7
:103EB00080B588B00690FFE7FFE70698006850E8F5
:103EC000030F20F4F0700590FFE70599069802684B
:103ED00042E803100028F0D1FFE7FFE7FFE7FFE724
:103EE0000698006850E8050F20F001000490FFE7F5
:103EF00004990698026842E805100028F0D1FFE70F
:103F0000FFE70698006B012814D1FFE7FFE7FFE702
:103F10000698006850E8030F20F010000390FFE7B8
:103F200003990698026842E803100028F0D1FFE7E1
:103F3000FFE7FFE70698006840690006002832D5D1
:103F4000FFE7FFE7FFE70698006850E8050F20F05D
:103F500080000290FFE702990698026842E8051087
:103F60000028F0D1FFE7FFE70698806BD0B1FFE7AC
:103F70000698816B002048630698806BFDF79CFAD9
:103F800078B1FFE70698806BFDF762FB202807D128
:103F9000FFE706991020486403208DF81F004EE0CB
:103FA000FFE7FFE7FFE70698006840694006002842
:103FB00032D5FFE7FFE7FFE70698006850E8050FF6
:103FC00020F040000190FFE701990698026842E85E
:103FD00005100028F0D1FFE7FFE70698C06BD0B1CD
:103FE000FFE70698C16B002048630698C06BFDF799
:103FF00063FA78B1FFE70698C06BFDF729FB20282C
:1040000007D1FFE706991020486403208DF81F00B0
:1040100015E0FFE7FFE7FFE706990020C88406994F
:10402000C88506994864069A202182F84210069AAB
:1040300082F84110069908638DF81F00FFE79DF88C
:104040001F0008B080BD000080B586B00490FFE777
:10405000FFE70498006850E8030F20F49070039085
:10406000FFE703990498026842E803100028F0D1A2
:10407000FFE7FFE7FFE7FFE70498006850E8050F58
:1040800020F001000290FFE702990498026842E8DC
:1040900005100028F0D1FFE7FFE70498006B012826
:1040A00014D1FFE7FFE7FFE70498006850E8030F2B
:1040B00020F010000190FFE701990498026842E89F
:1040C00003100028F0D1FFE7FFE7FFE7049800683E
:1040D00040694006002832D5FFE7FFE7FFE7049874
:1040E000006850E8050F20F040000090FFE70099BD
:1040F0000498026842E805100028F0D1FFE7FFE7C6
:104100000498C06BD0B1FFE70498C16B00204863EE
:104110000498C06BFDF7D0F978B1FFE70498C06B45
:10412000FDF796FA202807D1FFE70499102048648C
:1041300003208DF817000EE0FFE7FFE7FFE7049983
:104140000020C885049A202182F84210049908634F
:104150008DF81700FFE79DF8170006B080BD00003E
:1041600080B584B00290FFE7FFE70298006850E84E
:10417000030F20F0C0000190FFE701990298026848
:1041800042E803100028F0D1FFE7FFE7029800683B
:1041900040690006002832D5FFE7FFE7FFE70298F5
:1041A000006850E8050F20F080000090FFE70099BC
:1041B0000298026842E805100028F0D1FFE7FFE707
:1041C0000298806BD0B1FFE70298816B00204863B2
:1041D0000298806BFDF770F978B1FFE70298806B69
:1041E000FDF736FA202807D1FFE70299102048642E
:1041F00003208DF80F000CE0FFE7FFE7FFE70299CF
:104200000020C884029A202182F841108DF80F0006
:10421000FFE79DF80F0004B080BD000081B0009062
:1042200001B0704780B592B0119011980068006895
:10423000109011980068C0680F901198006840694C
:104240000E9000200D900C90109800F00F000D9033
:104250000D9888B9FFE79DF84000800600280AD530
:10426000FFE79DF83C008006002804D5FFE7119881
:1042700004F0B6FBE9E1FFE70D98002800F0C280EA
:10428000FFE79DF83800C00738B9FFE7BDF83C00EC
:1042900010F4907F00F0B680FFE79DF84000C00763
:1042A00058B1FFE79DF83D00C00730B1FFE7119915
:1042B000486C40F001004864FFE79DF8400040076B
:1042C00000280BD5FFE79DF83800C00730B1FFE7A5
:1042D0001199486C40F002004864FFE79DF84000E7
:1042E000800700280BD5FFE79DF83800C00730B1E4
:1042F000FFE71199486C40F004004864FFE79DF81F
:1043000040000007002811D5FFE79DF83C0080061B
:10431000002805D4FFE79DF83800C00730B1FFE75B
:104320001199486C40F008004864FFE71198406C10
:10433000002866D0FFE79DF84000800600280AD5D7
:10434000FFE79DF83C008006002804D5FFE71198A0
:1043500004F046FBFFE7119800684069C0F3801045
:104360000C901198406C0007002804D4FFE70C98CB
:1043700000283ED0FFE7119804F0D4FA11980068A5
:104380004069400600282FD5FFE7FFE7FFE71198B7
:10439000006850E8050F20F040000B90FFE70B99F4
:1043A0001198026842E805100028F0D1FFE7FFE706
:1043B0001198C06B98B1FFE71198C16B48F60510D2
:1043C000C0F6000048631198C06BFDF7B3F828B140
:1043D000FFE71198C06B416B8847FFE703E0119836
:1043E000FFF71CFFFFE703E01198FFF717FFFFE758
:1043F00006E01198FFF712FF119900204864FFE7CB
:10440000FFE722E11198006B012840F0FE80FFE7F2
:104410009DF84000C006002840F1F780FFE79DF8B6
:104420003C00C006002840F1F080FFE7FFE70020D5
:104430000A901198006800680A9011980068406816
:104440000A900A98FFE71198006840694006002822
:1044500040F18180FFE71198C06B00684068ADF8BB
:104460002600BDF82600002874D0FFE7BDF826001E
:104470001199898D88426DDAFFE7BDF82600119900
:10448000C8851198C06B8069202858D0FFE7FFE7E6
:10449000FFE71198006850E8030F20F4807008903F
:1044A000FFE708991198026842E803100028F0D14C
:1044B000FFE7FFE7FFE7FFE71198006850E8050F07
:1044C00020F001000790FFE707991198026842E881
:1044D00005100028F0D1FFE7FFE7FFE7FFE711989D
:1044E000006850E8050F20F040000690FFE70699AD
:1044F0001198026842E805100028F0D1FFE7FFE7B5
:104500001199202081F84200119900200863FFE7EB
:10451000FFE71198006850E8030F20F010000590A5
:10452000FFE705991198026842E803100028F0D1CE
:10453000FFE7FFE71198C06BFCF7BEFFFFE711999B
:10454000022048631198818DC28D891A89B2FFF7C4
:10455000A9FCFFE779E01199888DC98D401AADF863
:1045600012001198C08D00284ED0FFE7BDF8120050
:10457000002849D0FFE7FFE7FFE71198006850E8FF
:10458000030F20F490700390FFE7039911980268DD
:1045900042E803100028F0D1FFE7FFE7FFE7FFE75D
:1045A0001198006850E8050F20F001000290FFE725
:1045B00002991198026842E805100028F0D1FFE73F
:1045C000FFE71199202081F842001199002008632B
:1045D000FFE7FFE71198006850E8030F20F0100094
:1045E0000190FFE701991198026842E80310002842
:1045F000F0D1FFE7FFE71199022048631198BDF859
:104600001210FFF74FFCFFE71FE09DF84000000687
:1046100000280AD5FFE79DF83C000006002804D5D5
:10462000FFE7119804F022FB0FE09DF840004006E0
:1046300000280AD5FFE79DF83C004006002804D575
:10464000FFE7119804F0B8F9FFE712B080BD000051
:1046500080B582B00090009820B9FFE701208DF866
:10466000070040E00098806908B1FFE700E0FFE73D
:10467000009890F8410040B9FFE70099002081F8C8
:104680004000009800F034F8FFE70099242081F8FA
:10469000410000980168C86820F40050C860009884
:1046A00004F054FA00980168086920F49040086109
:1046B00000980168486920F02A0048610098016864
:1046C000C86840F40050C860009900204864009A0F
:1046D000202182F84110009A82F842100099486324
:1046E0008DF80700FFE79DF8070002B080BD0000CD
:1046F00080B592B01190002010900F900E900D9008
:104700001198006843F60001C4F20101884251D1BA
:10471000FFE7FFE741F21800C4F20200016841F42C
:1047200080410160006800F480400C900C98FFE725
:10473000FFE741F21800C4F20200016841F00801ED
:104740000160006800F008000B900B98FFE7402024
:104750000D9002200E900320109040F60040C4F20D
:10476000010006900DA90791FCF79AFF069807999A
:1047700080220D9200220E920F92FCF791FFFFE72C
:104780000421C4F2010108680A900A9840F0E06030
:104790000A900A9840F004000A900A980860FFE71F
:1047A0002520059000221146FDF7A4FB0598FDF792
:1047B00097FB4AE01198006844F20041C4F20001FE
:1047C000884241D1FFE7FFE741F21C00C4F202003A
:1047D000016841F400310160006800F40030099084
:1047E0000998FFE7FFE741F21800C4F202000168F0
:1047F00041F004010160006800F00400089008988E
:10480000FFE704200D9002200E900320109040F648
:104810000000C4F2010001900DA90291FCF740FFD5
:104820000198029908220D92002203920E920F9293
:10483000FCF736FF039A262004901146FDF75AFB39
:104840000498FDF74DFBFFE7FFE712B080BD0000C5
:1048500080B584B002900191ADF80220029890F8E2
:104860004200202817D1FFE7019820B1FFE7BDF8EB
:10487000020020B9FFE701208DF80F000FE0029938
:104880000020086302980199BDF8022004F0BCF9E9
:104890008DF80F0003E002208DF80F00FFE79DF870
:1048A0000F0004B080BD000081B0009001B07047DF
:1048B00084B002900191ADF80220029890F8410076
:1048C000202826D1FFE7019820B1FFE7BDF80200BC
:1048D00020B9FFE701208DF80F001EE00198029932
:1048E0000862BDF8020002998884BDF802000299AE
:1048F000C884029900204864029A212182F841105C
:1049000002990A68D16841F08001D1608DF80F00EA
:1049100003E002208DF80F00FFE79DF80F0004B0C0
:104920007047000081B0009001B07047FFE7FEE7DC
:1049300083B0ADF80800ADF80610ADF80420ADF86E
:104940000230BDF80800BDF80410884215DBFFE70F
:10495000BDF80800BDF80410401ABDF80610084460
:10496000BDF80210884204DDFFE702208DF80B003D
:1049700007E000208DF80B0003E002208DF80B000B
:10498000FFE79DF80B0003B07047000080B586B0CC
:1049900084460898CDF810C0ADF80E10ADF80C2084
:1049A00002938DF80700BDF80C00B0F5FA6F04DD36
:1049B000FFE703208DF8170027E0BDF80E00BDF8D3
:1049C0000C1000224FF47A73FFF7B2FF78B9FFE7BB
:1049D000BDF80E00C0F30B1140F27830C2F20000B7
:1049E00000EB410000F674100499086003E0022017
:1049F0008DF8170009E0BDF80E0000F00F000299D5
:104A0000088000208DF81700FFE79DF8170006B01A
:104A100080BD000080B584B00290ADF80610ADF8FE
:104A200004208DF80330BDF804007E2804DBFFE786
:104A300003208DF80F0049E09DF80300E8B9FFE777
:104A4000BDF80600BDF8041000224FF4FA63FFF72A
:104A50006FFF68B9FFE7BDF8061040F27830C2F288
:104A6000000000EB410000F6A6100299086003E088
:104A700002208DF80F0029E024E09DF803000128B2
:104A80001BD1FFE7BDF80600BDF8041000224FF46B
:104A9000FA63FFF74DFF58B9FFE7BDF8061040F283
:104AA0007830C2F2000000EB41000299086003E098
:104AB00002208DF80F0009E003E001208DF80F00BF
:104AC00004E0FFE700208DF80F00FFE79DF80F00DE
:104AD00004B080BD84B00390029100208DF80700DF
:104AE000009002984078082803D1FFE70120009049
:104AF00018E0029840782B2803D1FFE700200090AF
:104B00000FE00298407800F07F000E2803D8FFE7FE
:104B10000120009004E00298007B02300090FFE743
:104B2000FFE7FFE7009807300090009804B0704757
:104B300040F6C061C2F200010720086049F65250F9
:104B4000C0F60000486001228A6049F65850C0F65D
:104B50000000C8600A6148618A61C8610A624862EF
:104B60008A62C8627047000041F2C021C2F20001AF
:104B70000020088088708880C880088148818881EA
:104B8000C88108824882704741F2C021C2F2000108
:104B9000888801308880704741F2C020C2F200004E
:104BA000408A4FF6FE7188420CDCFFE741F2C021DB
:104BB000C2F20001488A01304882088840F00100B2
:104BC0000880FFE77047000041F2C020C2F20000F9
:104BD000C0884FF6FE71884208DCFFE741F2C02131
:104BE000C2F20001C8880130C880FFE770470000AA
:104BF00041F2C020C2F2000000894FF6FE718842E7
:104C000008DCFFE741F2C021C2F20001088901304F
:104C10000881FFE77047000041F2C020C2F20000A7
:104C200040894FF6FE71884208DCFFE741F2C0215F
:104C3000C2F20001488901304881FFE77047000057
:104C400041F2C020C2F20000C0894FF6FE718842D6
:104C500008DCFFE741F2C021C2F20001C88901303F
:104C6000C881FFE77047000041F2C020C2F2000097
:104C700080894FF6FE71884208DCFFE741F2C021CF
:104C8000C2F20001888901308881FFE77047000087
:104C900041F2C020C2F200008078704780B588B031
:104CA00006900591049200200390059800780499DD
:104CB000039A531C03938854059840780499039AE7
:104CC000531C03938854059890F90100002800F1C3
:104CD0008880FFE7059840782B2816D1FFE70598D4
:104CE00080780499039A531C039388540598C078DC
:104CF0000499039A531C0393885405988079049966
:104D0000039A531C039388546AE005984078082856
:104D10001DD1FFE70598C07B0499039A531C0393A8
:104D200088540598C0890499039A531C03938854A6
:104D30000598407C0499039A531C03938854059862
:104D4000008A0499039A531C0393885447E00598FA
:104D5000407A0499039A531C039388540598008958
:104D60000499039A531C039388540598C07A0499B4
:104D7000039A531C03938854059840890499039A15
:104D8000531C03938854059840780F2805D0FFE7FB
:104D900005984078102821D1FFE70598007B0499F9
:104DA000039A531C0393885405980E3002900020F8
:104DB0000190FFE701980599097B88420DDAFFE72A
:104DC00002980199405C0499039A531C03938854F8
:104DD000FFE7019801300190ECE7FFE7FFE7FFE70D
:104DE000FFE70398B0F1FF3F04DCFFE707208DF8F1
:104DF0001F001FE00498039903F0F4FFADF80200D0
:104E0000BDF802000599A1F80A01BDF80200049955
:104E1000039A531C039388549DF803000499039A42
:104E2000531C0393885403980699C86001208DF899
:104E30001F00FFE79DF81F0008B080BD80B58EB051
:104E40000C900B910A920020099008900A980999F9
:104E50004A1C0992405C0B9908700A9809994A1CEF
:104E60000992405C0B9948700B9840780006002826
:104E700009D5FFE70A9809994A1C0992405C0B99E9
:104E800081F808013BE10B9890F90100002800F13E
:104E90003581FFE70B9840782B287AD1FFE70A98F5
:104EA00009994A1C0992405C0B9988700A980999E3
:104EB0004A1C0992405C0B99C8700A9809994A1CCF
:104EC0000992405C0B9908710A9809994A1C099249
:104ED000405C0B9948710A9809994A1C0992405CF8
:104EE0000B9988710A9809994A1C0992405C0B99A0
:104EF000C8710B99002008730B990E310791069029
:104F00000590FFE705980B99C979884240DAFFE7D9
:104F10000A9809994A1C0992405C8DF813009DF883
:104F200013000799069A531C069388540A98099906
:104F30004A1C0992405C8DF812009DF812000799F6
:104F4000069A531C0693885400200390FFE70398A9
:104F50009DF8121088420FDAFFE70A9809994A1C57
:104F60000992405C0799069A531C06938854FFE700
:104F7000039801300390EAE79DF812000B990A7B31
:104F8000104402300873FFE7059801300590B9E737
:104F9000B3E00B984078082823D1FFE70A980999D5
:104FA0004A1C0992405C00020B99C8810A98099931
:104FB0004A1C0992425C0B99C8891043C8810A981F
:104FC00009994A1C0992405C00020B9908820A98D0
:104FD00009994A1C0992425C0B99088A104308827D
:104FE0008AE00B98407801280FD0FFE70B984078B3
:104FF00002280AD0FFE70B984078032805D0FFE786
:105000000B98407804283ED1FFE70A9809994A1C7A
:105010000992405C0B9908730B980E3002900020A7
:105020000190FFE701980B99097B88422ADAFFE794
:10503000019800EBD07121F00101401A70B9FFE72F
:105040000A9809994A1C0992405C00020299019A47
:1050500002EBD27222F0010288520EE00A980999FE
:105060004A1C0992435C0299019800EBD07020F031
:105070000102885A18438852FFE7FFE70198013080
:105080000190CFE737E00B98407805280FD0FFE775
:105090000B98407806280AD0FFE70B9840780F2835
:1050A00005D0FFE70B984078102823D1FFE70A9836
:1050B00009994A1C0992405C00020B9908810A98E0
:1050C00009994A1C0992425C0B990889104308818E
:1050D0000A9809994A1C0992405C00020B99488180
:1050E0000A9809994A1C0992425C0B994889104315
:1050F0004881FFE7FFE7FFE7FFE7FFE7FFE70A98E1
:10510000099903F06FFEADF802000A9809994A1C4C
:105110000992405C0B99A1F80A010A9809994A1C66
:105120000992425C0B99B1F80A0140EA0220A1F809
:105130000A010B98B0F80A01BDF80210884204D0A9
:10514000FFE708208DF8370003E001208DF83700D5
:10515000FFE79DF837000EB080BD000080B586B037
:1051600004900498C089ADF80E000498008AADF848
:105170000C0041F2C020C2F200008078012809D161
:10518000FFE7BDF80E00012804D0FFE700208DF8EE
:10519000170025E1BDF80E0001460291142800F227
:1051A0000E810299DFE811F0150021004C005B0030
:1051B00068000B010B010B010B010B0172007F005A
:1051C0008E009D00AC00BB00CA00D900E8000B01B6
:1051D000F700BDF80E000499C881BDF80C000499D1
:1051E0000882049904200873F6E041F2C021C2F25B
:1051F000000100208870BDF80C00B0F57F4F03D18E
:10520000FFE7FFF7B1FC0FE041F2C021C2F200015D
:105210000091002001908880C880088148818881A1
:10522000C88108824882FFE7BDF80E000499C88152
:10523000BDF80C0004990882049904200873CBE09F
:10524000BDF80E000499C88141F2C020C2F20000EE
:10525000008804990882049904200873BCE004992A
:10526000487840F0800048700499012081F80801D6
:1052700000208DF81700B3E041F2C021C2F2000116
:105280000120887000208DF81700A9E0FFF76CFC62
:10529000BDF80E000499C881049900200882049981
:1052A0000420087398E0BDF80E000499C88141F20B
:1052B000C020C2F20000808804990882049904206A
:1052C000087389E0BDF80E000499C88141F2C0203E
:1052D000C2F20000C088049908820499042008736F
:1052E0007AE0BDF80E000499C88141F2C020C2F2F4
:1052F00000000089049908820499042008736BE077
:10530000BDF80E000499C88141F2C020C2F200002D
:105310004089049908820499042008735CE0BDF870
:105320000E000499C88141F2C020C2F200008089B9
:10533000049908820499042008734DE0BDF80E001A
:105340000499C88141F2C020C2F20000C0890499CA
:1053500008820499042008733EE0BDF80E00049909
:10536000C88141F2C020C2F20000008A049908827C
:105370000499042008732FE0BDF80E000499C88139
:1053800041F2C020C2F20000408A049908820499C8
:105390000420087320E041F2C022C2F20002002083
:1053A0005082118821F001011180BDF80E10049A7D
:1053B000D181049908820499042008730CE00499AF
:1053C000487840F0800048700499012081F8080175
:1053D00000208DF8170003E001208DF81700FFE78B
:1053E0009DF8170006B080BD80B58AB008900020F7
:1053F000ADF81A00089A118952896B46186007A8FF
:105400000DF11A03FFF7C2FA089981F8080108980C
:1054100090F8080120B1FFE700208DF827008AE00E
:1054200008994889013800EB5072012000EBD20046
:1054300008730020ADF81800ADF81600ADF81400A0
:10544000ADF81200BDF81A1003910290FFE7029820
:10545000BDF81A10089A52891144013901EB1172F2
:10546000012101EB221188424EDCFFE70020ADF85C
:105470001800FFE703980F281ADCFFE703990120C3
:1054800000FA01F1BDF818000843ADF81800BDF8A6
:1054900012000130ADF8120080B2089949898842A3
:1054A00001DBFFE704E0FFE7039801300390E1E749
:1054B000002003900798029A30F81200BDF81810E7
:1054C0000840BDF81A10C840089901EB4201C88194
:1054D0000298012813DBFFE70798029930F81100C2
:1054E000BDF8182010400004BDF81A2040FA02F25E
:1054F000089800EB4101888910438881FFE7FFE7A6
:10550000029801300290A2E7FFE7029800280ED42B
:10551000FFE70898029900EB4101CA89100A40EAA6
:105520000220C881FFE7029801380290EDE70120D0
:105530008DF82700FFE79DF827000AB080BD000026
:1055400080B584B002900299822008710298C078D8
:10555000013801460191032831D80199DFE801F0B3
:10556000021222270298807920B9FFE702990020D1
:105570008871FFE70298022100F072FE0299032071
:10558000C87120E00298807920B9FFE702990320D2
:105590008871FFE70298062100F062FE029904205C
:1055A000C87110E00299032081F808010BE002980D
:1055B000817900F055FE02990120C87103E00020B6
:1055C0008DF80F000CE0029890F8080120B1FFE779
:1055D00000208DF80F0003E001208DF80F00FFE799
:1055E0009DF80F0004B080BD80B584B00290029891
:1055F0000189428901A80023FFF70CFA029981F87A
:105600000801029890F8080120B1FFE700208DF80A
:105610000F001EE0029948894000087300200090A6
:10562000FFE700980299498988420EDAFFE701985E
:10563000811C019100880299009A01EB4201C88106
:10564000FFE7009801300090EBE701208DF80F0094
:10565000FFE79DF80F0004B080BD000080B584B066
:10566000029002980189428901A80123FFF7D2F92B
:10567000029981F80801029890F8080120B1FFE72B
:1056800000208DF80F002FE0029948894000087330
:1056900000200090FFE700980299498988421FDAAC
:1056A000FFE70198B0F9000001280ADBFFE7019845
:1056B000811C019100880299009A01EB4201C88186
:1056C00009E00198811C019100880299009A01EB80
:1056D0004201C881FFE7FFE7009801300090DAE758
:1056E00001208DF80F00FFE79DF80F0004B080BD8A
:1056F00080B58AB008900899087B4989013901EB87
:105700005172012101EBE201884208D0FFE70899BC
:10571000032081F8080100208DF82700A2E0002076
:10572000ADF81A000898018942896B46012018607B
:1057300007A80DF11A03FFF729F9089981F8080164
:10574000089890F8080120B1FFE700208DF82700A5
:1057500088E00020ADF818000590ADF81200ADF813
:105760001000BDF81A1003910290FFE70298BDF8EF
:105770001A10089A52891144013901EB1172012162
:1057800001EB2211884269DCFFE70020ADF8180028
:10579000FFE703980F281ADCFFE70399012000FABE
:1057A00001F1BDF818000843ADF81800BDF810006D
:1057B0000130ADF8100080B208994989884201DBB8
:1057C000FFE704E0FFE7039801300390E1E70020E2
:1057D00003900798029930F81100ADF8120008986C
:1057E000029900EB4100C08940BABDF81A10884008
:1057F0000590029801280FDBFFE70898029900EB5B
:105800004100808940BABDF81A1000FA01F10598EC
:1058100040EA21400590FFE70598BDF818100840C0
:105820000799029A21F81200BDF81200BDF818106D
:1058300020EA01030799029A31F81200184321F86F
:105840001200BDF8100008994989884201DBFFE782
:1058500004E0FFE702980130029087E701208DF80D
:105860002700FFE79DF827000AB080BD80B584B00F
:10587000029002984189007BB0EB410F08D0FFE70E
:105880000299032081F8080100208DF80F002DE017
:1058900002980189428901A80023FFF7BBF8029909
:1058A00081F80801029890F8080120B1FFE7002074
:1058B0008DF80F001AE000200090FFE70098029991
:1058C000498988420EDAFFE70298009900EB41000F
:1058D000C08901998A1C01920880FFE70098013075
:1058E0000090EBE701208DF80F00FFE79DF80F0017
:1058F00004B080BD80B586B004900498408970B132
:10590000FFE704984089B0F57F4F08D0FFE704997E
:10591000032081F8080100208DF8170036E00022EE
:10592000ADF80A20049801896B460120186003A88D
:105930000DF10A03FFF72AF8049981F80801049889
:1059400090F8080120B1FFE700208DF817001DE056
:1059500004984089B0F57F4F0AD1FFE7BDF80A10DF
:10596000012000FA01F2039908881043088009E039
:10597000BDF80A10012000FA01F20399088890434B
:105980000880FFE701208DF81700FFE79DF817005A
:1059900006B080BD80B584B002900298018901A84C
:1059A00001220023FFF736F8029981F808010298D6
:1059B00090F8080120B1FFE700208DF80F0007E004
:1059C000029840890199088001208DF80F00FFE7B7
:1059D0009DF80F0004B080BD80B58AB00890079193
:1059E000069200200590089890F82100C00760B149
:1059F000FFE7089890F820100020B0EBD11F04D0EA
:105A0000FFE70898C0680590D4E0079800780699E9
:105A1000059A531C05938854079840780699059A6F
:105A2000531C05938854079890F90100002800F151
:105A3000B780FFE7079840782B284FD1FFE70798FA
:105A400080780699059A531C059388540798C07866
:105A50000699059A531C059388540798007906996E
:105A6000059A531C05938854079840790699059A1E
:105A7000531C05938854079880790699059A531CFE
:105A8000059388540798C0790699059A531C059385
:105A900088540798007BFB2804DBFFE707208DF87C
:105AA0002700B0E007980E30049000200390FFE735
:105AB00003980799097B88420FDAFFE7049800787A
:105AC0000699059A531C0593885404980130049054
:105AD000FFE7039801300390EAE760E00798407819
:105AE00008281DD1FFE70798C07B0699059A531C2B
:105AF000059388540798C0890699059A531C059305
:105B000088540798407C0699059A531C059388543D
:105B10000798008A0699059A531C059388543DE01E
:105B20000798007BFA2808DCFFE70798007B0699B6
:105B3000059A531C0593885403E007208DF827002D
:105B400061E007980E30029000200190FFE7019875
:105B50000799097B884220DAFFE7019800EBD071B2
:105B600021F00101401A40B9FFE7029840780699F8
:105B7000059A531C059388540AE002980078069908
:105B8000059A531C05938854029802300290FFE74F
:105B9000FFE7019801300190D9E7FFE7FFE708E050
:105BA000079890F808010699059A531C05938854A4
:105BB000FFE7FFE70598B0F1FF3F04DCFFE70720B0
:105BC0008DF827001FE00698059903F00BF9ADF852
:105BD0000200BDF802000799A1F80A019DF8020031
:105BE0000699059A531C059388549DF8030006995D
:105BF000059A531C0593885405980899C86001209C
:105C00008DF82700FFE79DF827000AB080BD00004F
:105C100080B58AB008900791069200200490089AF7
:105C200092F8201001F0BF0182F82010039006982E
:105C30000499405C08990978884207D0FFE70799E2
:105C40000020087004980130049007E00698049939
:105C50004A1C0492405C07990870FFE70698049973
:105C60004A1C0492405C07994870079840780006E7
:105C7000002809D5FFE7FEF7E3FF07990020087029
:105C800005208DF827001EE1079840782B2819D1B0
:105C9000FFE7069804994A1C0492405C07998870B3
:105CA000069804994A1C0492405C0799C8700698AB
:105CB00004994A1C0492405C079988710799002056
:105CC000087350E007984078082828D1FFE7069825
:105CD00004994A1C0492405C00020799C881069806
:105CE00004994A1C0492425C0799C8891043C881F0
:105CF000069804994A1C0492405C000207990882A5
:105D0000069804994A1C0492425C0799088A104339
:105D100008820799002008810799488122E00698A7
:105D200004994A1C0492405C000207990881069875
:105D300004994A1C0492425C07990889104308811F
:105D4000069804994A1C0492405C00020799488115
:105D5000069804994A1C0492425C079948891043AA
:105D60004881FFE7FFE70898406840780F2806D091
:105D7000FFE7089840684078102809D1FFE70698A7
:105D800004994A1C0492405C08994968087304E02D
:105D90000898416800200873FFE708980799FEF704
:105DA00099FE03900898C068039988420BDAFFE7D0
:105DB000089991F8200040F0400081F8200005206B
:105DC0008DF827007FE00898C0680399884206DDB7
:105DD000FFE7FEF7F9FE08208DF8270073E0FFE7E4
:105DE0000798007B002840D0FFE70798007BFB283E
:105DF0000BDBFFE70799487840F080004870FEF71A
:105E0000E3FE08208DF827005DE007980E30029031
:105E100000200190FFE701980799097B884223DA67
:105E2000FFE7019800EBD07121F00101401A48B959
:105E3000FFE7069804994A1C0492405C000202990C
:105E400008800CE0069804994A1C0492425C02996E
:105E5000088810430880029802300290FFE7FFE7AD
:105E6000019801300190D6E7FFE70698049902F007
:105E7000B9FFADF80200069804994A1C0492405CF0
:105E80000799A1F80A01069804994A1C0492425CF9
:105E90000799B1F80A0140EA0220A1F80A0107981F
:105EA000B0F80A01BDF80210884208D0FFE7FEF7FB
:105EB0008BFE0799487840F080004870FFE701208A
:105EC0008DF82700FFE79DF827000AB080BD00008D
:105ED00080B586B00490039100208DF80B000499E2
:105EE00091F8200000F07F0081F82000049991F8DB
:105EF000210000F0FE0081F82100049991F82000B3
:105F000000F0F70081F82000049991F8200000F0DB
:105F1000DF0081F82000FEF737FE0498007820B1FA
:105F2000FFE70398007868B9FFE7FEF79DFE049944
:105F3000052081F828000498039901F0F1F98DF803
:105F4000170088E1FEF768FE039890F90100002829
:105F500000F15181FFE70398407801380146019133
:105F60002A2800F21F810199DFE811F02B001C01A3
:105F70003A004900580082001C010D011C011C015F
:105F80001C011C011C011C01AC00D5001C011C01E2
:105F90001C011C011C011C011C011C011C011C0119
:105FA0001C011C011C011C011C011C011C011C0109
:105FB0001C011C011C011C011C011C011C011C01F9
:105FC000FE0004984068FFF70FFA0246049991F822
:105FD000200000F07F0040EAC21081F82000E6E0D7
:105FE00004984068FFF700FB0246049991F82000EE
:105FF00000F07F0040EAC21081F82000D7E004984A
:106000004068FFF72BFB0246049991F8200000F04E
:106010007F0040EAC21081F82000C8E00498406880
:10602000FFF768FC0246049991F8200000F07F0019
:1060300040EAC21081F82000049890F82010002057
:10604000B0EBD11F13D0FFE7049991F8210040F085
:10605000040081F82100049991F8210040F001002A
:1060600081F821000499C8680238C860FFE79EE003
:1060700004984068FFF78EFC0246049991F82000CE
:1060800000F07F0040EAC21081F82000049890F8E8
:1060900020100020B0EBD11F13D0FFE7049991F836
:1060A000210040F0040081F82100049991F82100BA
:1060B00040F0010081F821000499C8680238C860E6
:1060C000FFE774E004984068FFF712FB024604996A
:1060D00091F8200000F07F0040EAC21081F8200013
:1060E000049890F820100020B0EBD11F12D0FFE7E9
:1060F000049991F8210040F0040081F821000499EE
:1061000091F8210040F0010081F821000499062057
:10611000C860FFE74BE004984068FFF7A7FB024622
:10612000049991F8200000F07F0040EAC21081F845
:106130002000049890F820100020B0EBD11F12D05E
:10614000FFE7049991F8210040F0040081F8210054
:10615000049991F8210040F0010081F82100049990
:106160000620C860FFE722E004984068FFF7E8F9DE
:106170000246049991F8200000F07F0040EAC21026
:1061800081F8200013E004984068FEF7E7FF02461C
:10619000049991F8200000F07F0040EAC21081F8D5
:1061A000200004E00399012081F80801FFE7FEF7D1
:1061B0006FFD01280DD1FFE7FEF756FD049905207C
:1061C00081F828000498039901F0AAF88DF81700C7
:1061D00041E0049890F820100020B0EBD11F08D1C6
:1061E000FFE7FEF705FD0399487840F0800048700E
:1061F00000E0FFE7FFE7049890F82000C008C00720
:1062000028B1FFE70498012100F0CEFFFFE70498D2
:1062100090F821004008C00738B9FFE704980399B7
:1062200001F0B4F88DF80B000BE00498039901F02D
:1062300077F8049991F8210000F0FD0081F8210021
:10624000FFE79DF80B00049981F828009DF80B00EA
:106250008DF81700FFE79DF8170006B080BD00001D
:1062600080B58AB00990089140F6C060C2F2000083
:1062700007900998807906900999002081F8080113
:1062800005900490FFE70498F9281EDCFFE70698C4
:10629000FF2801D3FFE718E0049802300490079824
:1062A000069950F831100498084404900498F9288D
:1062B00004DCFFE7069801300690FFE7069808998E
:1062C000884201D9FFE700E0DDE706980138059034
:1062D00009980E300390002002900998807901906F
:1062E000FFE701980599884213D8FFE701980399C1
:1062F000029A531C0293885403980799019A01EB60
:10630000C20202A900F028F8FFE7019801300190CD
:10631000E7E70198013801900998007BA8B1FFE7F1
:1063200002980999087305980130099988710198B4
:106330000899884204D1FFE709990020487103E0D9
:106340000999FF204871FFE704E00999032081F8CB
:106350000801FFE70AB080BD84B00390029101926A
:10636000019800680399DDF808C0DCF80020531C90
:10637000CCF80030885400200090FFE70098019985
:106380000968884212D2FFE7019840680099405C92
:106390000399DDF808C0DCF80020531CCCF800306D
:1063A0008854FFE7009801300090E7E704B0704799
:1063B00084B002908DF80710ADF804208DF80330FA
:1063C000029820B9FFE701208DF80F002EE09DF81C
:1063D000030098B9FFE79DF80700012805DBFFE7F8
:1063E0009DF80700F82804DBFFE701208DF80F0077
:1063F0001CE09DF807000299087003E00299002054
:106400000870FFE7BDF80400029948839DF8030077
:1064100020B1FFE702990320087603E002990120EA
:106420000876FFE700208DF80F00FFE79DF80F00CA
:1064300004B0704780B584B0029001910092029838
:1064400018B1FFE7019820B9FFE701208DF80F0090
:1064500022E0FEF76DFB029903200870029941F2D9
:106460008830488302990120087602980199009AA1
:10647000002300F0B3FF029981F82800029890F8F9
:106480002800012804D1FFE700208DF80F0003E069
:1064900001208DF80F00FFE79DF80F0004B080BDCC
:1064A00080B584B002900191029820B9FFE70120E5
:1064B0008DF80F002EE00298007E032804DBFFE732
:1064C00001208DF80F0025E0FEF74EFB019840B14A
:1064D000FFE70298019900F0CFFF029981F82800A8
:1064E0000AE0029841F2D421C2F2000100F0C4FF98
:1064F000029981F82800FFE7029890F82800012807
:1065000004D1FFE700208DF80F0003E001208DF893
:106510000F00FFE79DF80F0004B080BD80B584B088
:10652000002203920292019241F2F850C2F200005E
:10653000009042F20041C4F2010101608260012139
:10654000017302754FF46023C36142600161FAF781
:106550004FFD18B1FFE7FAF7F9FBFFE711200190B3
:10656000012002900020039041F2F850C2F2000096
:1065700001A9FAF763FC18B1FFE7FAF7E7FBFFE7B9
:1065800004B080BD80B582B041F22860C2F2000044
:10659000009046F20041C4F2000101601021416008
:1065A000002101918160C160016141610176417604
:1065B0008176C17601774177FAF742FE18B1FFE79D
:1065C000FAF7C4FBFFE702B080BD000080B592B0CF
:1065D0000020119010900F900E90FFE741F21800EC
:1065E000C4F20200016841F010010160006800F08F
:1065F00010000D900D98FFE7FFE741F21800C4F27C
:106600000200016841F020010160006800F02000F4
:106610000C900C98FFE7FFE741F21800C4F202006B
:10662000016841F004010160006800F004000B9073
:106630000B98FFE7FFE741F21800C4F2020001687F
:1066400041F008010160006800F008000A900A9813
:10665000FFE741F20000C4F2010001904FF4005145
:10666000009100220592FBF7ABF9059A40F6000075
:10667000C4F20100029048F2F2710391FBF7A0F915
:10668000059A40F60040C4F2010007904FF607411A
:106690000991FBF795F9009A019805990E9201224C
:1066A00004920F9210910221069111910EA9089166
:1066B000FAF7F6FF0298049B059A08990E930F9239
:1066C0001092FAF7EDFF0298DDF810C0059B069ACC
:1066D0000899DDF80CE0CDF838E0CDF83CC0109317
:1066E0001192FAF7DDFFDDF810C0059B069A0798B6
:1066F0000899DDF824E0CDF838E0CDF83CC01093DF
:106700001192FAF7CDFF12B080BD000080B582B0C3
:1067100041F26460C2F20000019045F20041C4F20F
:106720000001016048F2A061C0F201014160002156
:106730008160C1604FF48042026141618161C16149
:106740000162FBF75BF918B1FFE7FAF7FFFAFFE721
:1067500002B080BD80B584B000208DF80E00ADF889
:106760000C0002908DF8070041F61C00C2F20000F8
:1067700042F60001C4F2000101604FF0FF314160B8
:106780004FF440718160FCF749FC18B1FFE7FAF75C
:10679000DDFAFFE701F080FD8DF807009DF80700A6
:1067A00068BBFFE700228DF80C208DF80D208DF8D6
:1067B0000E2041F61C00C2F2000003A9FCF7B4FD54
:1067C00018B1FFE7FAF7C2FAFFE701208DF80800D9
:1067D0008DF809008DF80A0000228DF80B2041F693
:1067E0001C00C2F2000002A9FCF7DEFC18B1FFE7B2
:1067F000FAF7ACFAFFE702A801F0A6FDFFE704B044
:1068000080BD000080B582B041F63000C2F20000C9
:10681000019043F20001C4F2010101604FF4827162
:10682000416000218160C160016141614FF40072EB
:1068300082610822C2610162416281620A21C162F1
:10684000FCF746FE18B1FFE7FAF780FAFFE702B05F
:1068500080BD000080B588B00021009107910691AD
:10686000059104910391029141F68800C2F2000063
:10687000019042F60042C4F2010202604160816070
:106880004FF6FF72C260016141618161FCF770FFE8
:1068900018B1FFE7FAF75AFAFFE74FF48050049077
:1068A00041F68800C2F2000004A9FDF709F918B109
:1068B000FFE7FAF74BFAFFE700200290039041F65A
:1068C0008800C2F2000002A9FCF7E4FE18B1FFE75D
:1068D000FAF73CFAFFE708B080BD000080B588B049
:1068E0000021019107910691059104910391029174
:1068F00041F6D000C2F200004FF08042026041F643
:106900001F42426081604FF6FF72C2600161816187
:10691000FCF72EFF18B1FFE7FAF718FAFFE74FF47C
:106920008050049041F6D000C2F2000004A9FDF7A7
:10693000C7F818B1FFE7FAF709FAFFE7002002905D
:10694000039041F6D000C2F2000002A9FCF7A2FEBB
:1069500018B1FFE7FAF7FAF9FFE708B080BD0000C9
:1069600080B588B0002101910791069105910491AD
:106970000391029141F66010C2F2000040F600025D
:10698000C4F20002026041F61F42426081604FF68D
:10699000FF72C26001618161FCF7EAFE18B1FFE796
:1069A000FAF7D4F9FFE74FF48050049041F66010F5
:1069B000C2F2000004A9FDF783F818B1FFE7FAF767
:1069C000C5F9FFE700200290039041F66010C2F283
:1069D000000002A9FCF75EFE18B1FFE7FAF7B6F96E
:1069E000FFE708B080BD000080B582B041F6A81076
:1069F000C2F2000001900121016343F60001C4F2DC
:106A0000010101604FF4E131416000218160C1600A
:106A100001610C2242618161C161FDF719FE18B16B
:106A2000FFE7FAF793F9FFE702B080BD80B582B0C7
:106A300041F6F010C2F2000001900121016344F21E
:106A40000041C4F2000101604FF4E13141600021D6
:106A50008160C16001610C2242618161C161FDF709
:106A6000F7FD18B1FFE7FAF771F9FFE702B080BD53
:106A7000FFE7FEE7FFE7FEE788B007900691059283
:106A8000079800F0070004900498C0F1070005285B
:106A900003D3FFE70420019004E00498C0F107004D
:106AA0000190FFE70198039004980430062803D86A
:106AB000FFE70020009003E0049803380090FFE710
:106AC0000098029006980399012202FA01F1013917
:106AD0000840029B984005999A40013A11400843AA
:106AE00008B0704783B002908DF8071000208DF831
:106AF0000600FFE79DF80700411E8DF80710A0B3C0
:106B0000FFE70298411C029100788DF805000820EB
:106B10008DF80400FFE79DF8040028B3FFE79DF817
:106B200006009DF80510484000F001008DF80300B4
:106B30009DF8060040088DF806009DF803209DF89A
:106B4000060080F08C01002A18BF08468DF8060068
:106B50009DF8050040088DF80500FFE79DF804004A
:106B600001388DF80400D6E7C4E79DF8060003B0AD
:106B70007047000086B00590059840F20C21C2F2E3
:106B8000000109684843049042F62440C4F2010021
:106B90000068ADF80E0000200290BDF80E00ADF8C0
:106BA0000600FFE702980499884218D2FFE742F6F0
:106BB0002440C4F201000068ADF80400BDF80400F0
:106BC000BDF80610401AADF80200BDF80210029898
:106BD00008440290BDF80400ADF80600E2E706B0F4
:106BE0007047000083B00290019100208DF80300EF
:106BF000FFE79DF8030007280EDCFFE702989DF8E9
:106C000003201044C07801998854FFE79DF80300E1
:106C100001308DF80300ECE703B0704780B584B015
:106C2000039003980121019100F05CF80199039809
:106C300000F042F84FF47A700090FFF79BFF039842
:106C40000021029100F038F80098FFF793FF0199B6
:106C5000039800F031F84FF4FA60FFF78BFF0298C9
:106C60000399087003998870039948700399C87252
:106C700004B080BD80B584B0039002910398552183
:106C800000F04EFA00208DF80700FFE79DF807009E
:106C900007280EDCFFE7039802999DF80720895C1E
:106CA00000F03EFAFFE79DF8070001308DF807007D
:106CB000ECE704B080BD000082B001908DF80310B5
:106CC0009DF8030028B1FFE70199888909690861E7
:106CD00005E001998889000409690861FFE702B0AD
:106CE0007047000083B002908DF807100298006989
:106CF0000430009040F20820C2F2000001680F202A
:106D000000FA01F200990868904308609DF80700B6
:106D100098B9FFE740F20820C2F20000016808209D
:106D200000FA01F2009908681043086002980169AE
:106D3000C86840F40040C8600CE040F20820C2F28D
:106D400000000168022000FA01F20099086810436F
:106D50000860FFE703B0704781B0009000980069B9
:106D60008068009989890840002818BF012001B077
:106D70007047000080B586B00390039820B9FFE704
:106D800000208DF8130026E0EFF3108072B6059016
:106D9000002101918DF80B100398FFF78DFF0398E8
:106DA0000121FFF79FFF0220FFF7E4FE01990398FE
:106DB000FFF798FF0620FFF7DDFE0398FFF7CCFFF3
:106DC0008DF80B003220FFF7D5FE62B69DF80B0060
:106DD0008DF81300FFE79DF8130006B080BD00009A
:106DE00080B584B00290029820B9FFE700208DF8AA
:106DF0000F0022E000208DF8070008208DF8060023
:106E0000FFE79DF80600411E8DF8061080B1FFE7F0
:106E10009DF8070040088DF807000298FFF7AAFFC9
:106E200001469DF8070040EAC1108DF80700E8E729
:106E30009DF807008DF80F00FFE79DF80F0004B0E4
:106E400080BD000080B584B00290029820B9FFE7B1
:106E500001208DF80F0021E0029800210091FFF73A
:106E60002BFF02980121FFF73DFF4FF4F070FFF771
:106E700081FE00990298FFF735FF4620FFF77AFE62
:106E80000298FFF769FF8DF807004FF4CD70FFF708
:106E900071FE9DF807008DF80F00FFE79DF80F00C9
:106EA00004B080BD80B586B004908DF80F100498B2
:106EB00020B9FFE700208DF81700E6E001208DF8EB
:106EC0000E0000218DF80D108DF80C108DF80B10B0
:106ED0008DF80A0004988078002840F0BF80FFE712
:106EE0000498FFF7AFFF50B1FFE704990020087046
:106EF00004998870049948708DF81700C5E00498CB
:106F00009DF80F1000F00CF9FFE70498FFF732FF2F
:106F10008DF809000498FFF72DFF8DF808009DF803
:106F20000900012806D1FFE79DF80800012801D1DA
:106F3000FFE77DE09DF809009DF80810884205D024
:106F4000FFE79DF809008DF8070034E09DF80E007A
:106F50000499097888420FDAFFE704989DF80C102D
:106F60000844C0789DF80A10014000200029C8BFDD
:106F700001208DF807000AE09DF80E0004990978B9
:106F8000401AB0FA80F040098DF80700FFE79DF83D
:106F9000070078B9FFE79DF80E008DF80D009DF809
:106FA0000D00082805DCFFE79DF80D0004994870E6
:106FB000FFE7FFE7FFE79DF8070001280AD1FFE799
:106FC0009DF80A2004989DF80C100144C8781043DD
:106FD000C87009E09DF80A2004989DF80C1001443F
:106FE000C8789043C870FFE704989DF8071000F038
:106FF00051F89DF80E0001308DF80E009DF80A0042
:1070000040008DF80A009DF80A0048B9FFE79DF896
:107010000C0001308DF80C0001208DF80A00FFE70C
:10702000FFE7FFE79DF80C000828FFF66EAFFFE7CB
:107030009DF80E00412810DBFFE79DF80D00049934
:1070400008700498007820B9FFE70499012088703F
:10705000FFE701208DF80B00FFE7FFE79DF80B002D
:1070600020B1FFE70498C07850B9FFE704990020E9
:10707000087004998870049948708DF80B00FFE738
:107080009DF80B008DF81700FFE79DF8170006B07C
:1070900080BD000080B586B004908DF80F10049874
:1070A00008B9FFE73AE0EFF3108072B605909DF85B
:1070B0000F00C0B1FFE7049800210291FFF7FCFD2B
:1070C00004980121FFF70EFE0820FFF753FD0299F7
:1070D0000498FFF707FE3220FFF74CFD0299049851
:1070E000FFF700FE18E0049800210191FFF7E4FD8E
:1070F000049801210091FFF7F5FD3920FFF73AFDD3
:1071000001990498FFF7EEFD0098FFF733FD019910
:107110000498FFF7E7FDFFE762B6FFE706B080BD22
:1071200080B582B001908DF80310019808B9FFE78F
:1071300017E008208DF80200FFE79DF80200411ECD
:107140008DF8021068B1FFE701989DF8031001F077
:107150000101FFF79FFF9DF8030040088DF8030031
:10716000EBE702B080BD00007047000082B00190E4
:10717000019840F20001C2F200010968C90844F612
:10718000D352C1F26202A1FB022189094843009057
:10719000FFE700BFFFE70098411E00910028F8D1EB
:1071A000FFE702B07047000080B584B003908DF80F
:1071B0000B1000208DF80A00039800F041FA9DF8AA
:1071C0000B004007002844D4FFE79DF80B00800720
:1071D000002823D5FFE703980069FCF735FF8DF8F9
:1071E0000A00039991F8200000F0FD0081F82000CA
:1071F000039991F8200000F0BF0081F82000039966
:1072000091F8200000F0FB0081F82000039991F82C
:10721000200000F0EF0081F82000FFE79DF80B0050
:10722000C007A8B1FFE703980069FCF799FF8DF844
:107230000A00039991F8200000F0F70081F820007F
:10724000039991F8200000F0DF0081F82000FFE7AB
:1072500042E003980069FCF72BFE8DF80A0000203D
:107260000190FFE70198B0F5817F0ADCFFE7039802
:107270008168019A00208854FFE70198013001904D
:10728000F0E7039991F8200000F0FD0081F820005C
:10729000039991F8200000F0BF0081F820000399C5
:1072A00091F8200000F0FB0081F82000039991F88C
:1072B000200000F0EF0081F82000039991F82000F1
:1072C00000F0F70081F82000039991F8200000F009
:1072D000DF0081F82000FFE70399032081F82800F0
:1072E00004B080BD80B584B00290019100920298F4
:1072F000007E022808DCFFE702980199009AFEF759
:107300006BFB8DF80F0007E002980199009AFDF7DA
:10731000C5FC8DF80F00FFE79DF80F0004B080BD9D
:1073200080B584B00390029100208DF80700039887
:10733000007E0146009101280CD0FFE7009802284A
:107340000FD0FFE70098032816D1FFE7039800F05D
:1073500051F9FFE70398029900F08EF88DF80700C5
:107360000AE0039991F8200000F0FE0081F8200067
:1073700001208DF80700FFE79DF80700012801D0E4
:10738000FFE7FFE79DF8070004B080BD80B584B03B
:107390000390029100208DF807000398007E0138C9
:1073A000022807D8FFE70398029900F079F98DF8D1
:1073B0000700FFE79DF8070001280BD0FFE70398BF
:1073C000007E022805DCFFE703980299FFF7A8FF7B
:1073D000FFE7FFE79DF8070004B080BD85B003908C
:1073E000029101920093039820B9FFE702208DF8E3
:1073F00013001FE0029820B9FFE702208DF8130068
:1074000018E002980399086101980399486103986C
:10741000806838B9FFE7039941F2F430C2F2000006
:10742000886003E0009803998860FFE701208DF8E9
:107430001300FFE79DF8130005B0704780B584B0D6
:107440000290019100920298007E022808DCFFE77A
:1074500002980199009AFEF7DBFB8DF80F0007E018
:1074600002980199009AFDF7E9FC8DF80F00FFE7FB
:107470009DF80F0004B080BD80B584B002900191EA
:1074800000208DF803008DF80200029890F820008B
:107490008008C00720B1FFE704208DF80F004DE001
:1074A000029991F8200040F0010081F82000029933
:1074B00091F8200040F0040081F82000029991F832
:1074C000200000F0EF0081F8200001980299486048
:1074D000029890F820008009C00720B9FFE70299C0
:1074E0000020C860FFE7029800690168C86840F0A2
:1074F0001000C86002988168C2680069114440F2B7
:107500000312FDF7A5F98DF802009DF8020038B1CD
:10751000FFE702980421FFF747FE8DF8030003E020
:1075200001208DF80300FFE79DF80300029981F820
:1075300028009DF803008DF80F00FFE79DF80F006D
:1075400004B080BD80B584B0029001910298007EA5
:10755000032804DBFFE702208DF80F0006E0029805
:107560000199FEF7B5FC8DF80F00FFE79DF80F00BD
:1075700004B080BD80B582B001900198406908B91F
:10758000FFE734E001984069FCF760FB01980421B3
:10759000FFF70AFE0199062081F828000198007E75
:1075A000022809DCFFE701994868007809788842D9
:1075B00001D1FFE7FFE7FFE70198007E032811DB19
:1075C000FFE7019991F8200000F0FE0081F820000B
:1075D0000198C06928B1FFE701984168C2699047E6
:1075E000FFE704E001984168FFF79AFEFFE702B069
:1075F00080BD000080B582B0019001984069D8B18B
:10760000FFE7019840690168002048620198408BBB
:1076100088B1FFE70199488B49690968C8620198F8
:107620004069FCF7CBF9019991F8200040F0020085
:1076300081F82000FFE7FFE7012002B080BD0000D5
:1076400080B582B0019001984069A8B1FFE7019828
:10765000408B28B1FFE701984069FCF707FAFFE784
:1076600001984069016800204862019840690168FA
:107670006FF001000861FFE7012002B080BD00004B
:1076800081B000900098406930B1FFE700984069F0
:10769000016800204862FFE7012001B07047000048
:1076A00080B584B00290019100208DF803008DF820
:1076B0000200029890F82000C008C00720B1FFE740
:1076C00004208DF80F005DE0029801998268FFF7B1
:1076D00009FE8DF803009DF80300012809D0FFE79B
:1076E00002980421FFF760FD02984168FFF718FE39
:1076F0003EE0029991F8200040F0010081F820005E
:10770000029991F8200040F0080081F820000299C9
:1077100091F8200000F0DF0081F820000198029924
:1077200048600298C06800280ADCFFE7029804213C
:10773000FFF73AFD8DF8030002208DF80F0021E0DD
:10774000029A916810699289FDF7B2F88DF80200EB
:107750009DF8020038B1FFE702980421FFF724FDED
:107760008DF8030003E001208DF80300FFE7FFE739
:107770009DF80300029981F828009DF803008DF818
:107780000F00FFE79DF80F0004B080BD80B582B008
:1077900001900198006908B9FFE700E1019991F8AB
:1077A000210040F0080081F821000198006900687C
:1077B0000068C006002840F1A580FFE70198006935
:1077C0000068C068C006002840F19C80FFE7FFE722
:1077D00000200090019800690068006800900198FE
:1077E00000690068406800900098FFE70198006910
:1077F000FCF718FD019991F8200000F0BF0081F816
:107800002000019890F820008008C007002878D058
:10781000FFE7019890F820004008C007002870D0CA
:10782000FFE701980169888DC98D421A0199C868DE
:107830001044C8600198C068012861DBFFE7019827
:107840000069FCF701FC019991F8200000F0FD00AF
:1078500081F82000019991F8200000F0BF0081F824
:107860002000019991F8200000F0FB0081F8200031
:10787000019991F8200000F0EF0081F820000199B3
:1078800091F8200040F0100081F820000198416834
:107890008268FFF7D3FD019981F82800019890F8DC
:1078A0002800012826D1FFE70198FFF7C9FE42F220
:1078B0006C40C2F200000068019948620198007EA5
:1078C000022805DCFFE701984168FFF73BFE10E066
:1078D000019991F8200000F0FE0081F82000019845
:1078E000C06928B1FFE701984168C2699047FFE786
:1078F000FFE704E001984168FFF712FDFFE7FFE7AB
:10790000FFE74CE001980069FCF78CFCFFE7019869
:107910000069406C80BBFFE701980069C08D0130B1
:1079200001990969898D88420BD1FFE7019890F888
:1079300020008008C00720B1FFE70198FFF75AFE3A
:10794000FFE70198FFF79CFE01980069C08C90B991
:10795000FFE7019890F82000C008C00758B1FFE782
:107960000198006990F84100212804D0FFE70198B0
:1079700000F018F8FFE712E001980069406C00077A
:10798000002803D5FFE7FDF707F9FFE70198042179
:10799000FFF70AFC01984168FFF7C2FCFFE702B05D
:1079A00080BD000080B582B0019001208DF80300F9
:1079B00000208DF80200019991F8200000F0F700F6
:1079C00081F82000019991F8200000F0DF0081F893
:1079D0002000019991F8200040F0200081F820005B
:1079E00001984168FFF79CFC8DF803009DF80300A7
:1079F00002B080BD82B08DF80700002000909DF895
:107A00000700000900EB80004000009000989DF8FE
:107A1000071001F00F010844C0B202B07047000027
:107A200082B08DF8070000200090FFE79DF8070066
:107A30000A2809D3FFE70098013000909DF807005D
:107A40000A388DF80700F1E7009800F00F019DF863
:107A5000070040EA011002B07047000080B584B012
:107A6000029000208DF80600ADF804000090029806
:107A700020B9FFE701208DF80F0040E041F61C001F
:107A8000C2F2000069460022FBF7A4F920B1FFE72B
:107A900001208DF80F0032E041F61C00C2F2000018
:107AA00001A90022FBF7E4F920B1FFE701208DF8DE
:107AB0000F0024E0684600F047FC9DF8040002999E
:107AC00008809DF80500029948809DF806000299FB
:107AD00088809DF802000299C8809DF801000299F3
:107AE00008819DF8030000F5FA60029948819DF82D
:107AF00000000299888100208DF80F00FFE79DF8B3
:107B00000F0004B080BD000080B584B002900298E0
:107B100020B9FFE700208DF80F0025E002980188CA
:107B200000201729019019D8FFE70298418800200A
:107B30003B29019012D8FFE70298818800203B2959
:107B400001900BD8FFE7029948898A79097A00F0F9
:107B5000C1F9002818BF01200190FFE7019800F04B
:107B600001008DF80F00FFE79DF80F0004B080BD05
:107B700080B586B0049000208DF80E00ADF80C00A2
:107B800002908DF80700049828B1FFE70498FFF7EA
:107B9000BBFF20B9FFE701208DF8170049E00498EA
:107BA00040890DF1070100F0CDFA20B9FFE701206F
:107BB0008DF817003DE0049800788DF80C000498CB
:107BC00080788DF80D00049800798DF80E009DF8EE
:107BD00007008DF80B000498007A8DF809000498CE
:107BE00080798DF80A0001208DF8080041F61C000C
:107BF000C2F2000003A90022FBF796FB20B1FFE7C9
:107C000001208DF8170014E041F61C00C2F20000BC
:107C100002A90022FBF7C8FA20B1FFE701208DF886
:107C2000170006E002A800F08FFB00208DF8170077
:107C3000FFE79DF8170006B080BD000080B586B054
:107C40000590049100200390029001900090059906
:107C5000C97B03910599497B02910599897B019123
:107C60000090FFE700980499884280F08C80FFE73D
:107C70000298012818D0FFE70298032814D0FFE7E4
:107C80000298052810D0FFE7029807280CD0FFE7DC
:107C90000298082808D0FFE702980A2804D0FFE7D6
:107CA00002980C281BD1FFE701981E2804D8FFE793
:107CB00001980130019011E002980C2806D0FFE7EE
:107CC0000298013002900120019006E0012002900C
:107CD0000190039801300390FFE7FFE74EE0029820
:107CE00004280CD0FFE70298062808D0FFE7029886
:107CF000092804D0FFE702980B280FD1FFE701986D
:107D00001D2804D8FFE701980130019005E0029892
:107D10000130029001200190FFE72EE00298022836
:107D20002AD1FFE701981B2804D8FFE7019801300A
:107D3000019020E001981C2811D1FFE7BDF80C004C
:107D400000F014F920B1FFE701980130019005E03F
:107D500002980130029001200190FFE70AE00198AB
:107D60001D2806D1FFE70298013002900120019002
:107D7000FFE7FFE7FFE7FFE7FFE7FFE7FFE7009821
:107D8000013000906EE703980599C8730298059931
:107D9000487301980599887303989DF808109DF819
:107DA000042000F01DFB0599087306B080BD00009B
:107DB00080B582B0ADF804008DF803109DF8030083
:107DC00028B1FFE79DF803000D2804D3FFE700204A
:107DD0008DF807001AE09DF8030002280AD1FFE79A
:107DE000BDF8040000F0FEF820B1FFE71D208DF87B
:107DF00007000BE09DF8030049F64651C0F600016C
:107E0000084410F8010C8DF80700FFE79DF8070003
:107E100002B080BD80B584B0029000200190F9F7D7
:107E2000E7FD0190FFE7029800684068800600289F
:107E30000DD4FFE7F9F7DCFD0199401AB0F57A7F20
:107E400004D9FFE703208DF80F000AE0EBE7029862
:107E50000168486840F01000486000208DF80F006D
:107E6000FFE79DF80F0004B080BD000080B584B02E
:107E700002900020019002980168486820F01000EC
:107E80004860F9F7B5FD0190FFE702980068406887
:107E9000800600280DD4FFE7F9F7AAFD0199401AE2
:107EA000B0F57A7F04D9FFE703208DF80F0004E0D6
:107EB000EBE700208DF80F00FFE79DF80F0004B0FE
:107EC00080BD000080B541F61C00C2F20000FAF748
:107ED0003BFF80BD80B584B0ADF80C008DF80B1071
:107EE0008DF80A2000208DF80900BDF80C10ADF8BF
:107EF00006108DF80500BDF80C000DF1090100F029
:107F000021F920B9FFE700208DF80F0029E0BDF826
:107F10000C00632807D8FFE7BDF80C0000F5FA60F5
:107F2000ADF80600FFE7BDF806009DF80B10FFF75F
:107F30003FFF8DF805009DF80A100020009051B118
:107F4000FFE79DF80A109DF8052000209142D8BF58
:107F500001200090FFE7009800F001008DF80F006D
:107F6000FFE79DF80F0004B080BD000081B0ADF8C0
:107F700000009DF80000800720B1FFE700208DF889
:107F800003002BE0BDF8000045F62941CCF28F211B
:107F900048434FEAB00045F62941C0F28F2188429C
:107FA00004D3FFE701208DF8030017E0BDF80000BF
:107FB00045F62941CCF28F2148434FEA30104DF26B
:107FC0000A71C0F2A301884204D8FFE701208DF8AE
:107FD000030003E000208DF80300FFE79DF8030095
:107FE00001B0704783B0ADF80A0000209DF80A1078
:107FF0008907019041BBFFE7BDF80A10012045F653
:108000002942CCF28F2251434FEAB10145F6284272
:10801000C0F28F229142009013D8FFE7BDF80A000A
:1080200045F62941CCF28F2148434FEA30114DF2F9
:108030000B72C0F2A3020020914238BF01200090D1
:10804000FFE700980190FFE7019800F0010003B0FE
:108050007047000080B588B007900020ADF8180088
:10806000059004900390ADF80A008DF80900079878
:1080700008B9FFE763E00798B0F8460BADF80A00CF
:108080000798B0F8440B012825D1FFE7079800F6C0
:10809000363003A9019100F09FF80198079A00215A
:1080A000A2F8441BFFF730FD20B9FFE70220ADF82E
:1080B0000A000FE003A8FFF75BFD20B1FFE70320F4
:1080C000ADF80A0005E00120ADF80A008DF80900BE
:1080D000FFE7FFE7FFE703A8FFF7C0FC40B1FFE7BA
:1080E00007990320A1F872090799A1F8460B26E029
:1080F000079800F6621003A9002200F009FA41F681
:108100008D20C2F20000007820B1FFE79DF8090041
:1081100078B1FFE7079800F63630BDF80A2003A9CA
:1081200000F0F6F941F68D21C2F20001012008703D
:1081300005E0BDF80A000799A1F8460BFFE708B073
:1081400080BD000082B0ADF804000091BDF80400CD
:10815000632808D8FFE79DF8040000990870012003
:108160008DF807001AE0BDF80400B0F5FA6F11D3DE
:10817000FFE7BDF8040040F6330188420AD8FFE764
:10818000BDF80400A0F5FA600099087001208DF890
:10819000070003E000208DF80700FFE79DF80700C7
:1081A00002B0704782B001900020ADF80200ADF837
:1081B000000001980068006AADF8020001980068AC
:1081C000406AADF80000BDF80210BDF8000040EABA
:1081D000014002B07047000082B001900091019808
:1081E00018B1FFE7009808B9FFE71CE00198008884
:1081F00000990880019840880099488001988088FB
:10820000009988800198C0880099C88001980089E9
:1082100000990881019840890099488101988089D6
:1082200000998881FFE702B07047000084B0039096
:108230000020ADF80A00ADF80800ADF80600009087
:10824000039800688069ADF80A0003980068C06967
:10825000ADF80600039800688069ADF80800BDF825
:108260000A00BDF8081088420AD0FFE7BDF80810E0
:1082700003980068C06980B240EA0140009007E0BE
:10828000BDF80A10BDF8060040EA01400090FFE783
:10829000009804B07047000080B586B000200490BC
:1082A0000390029041F61C00C2F200000121FAF78F
:1082B00015FD43F2A521884204D0FFE700208DF888
:1082C00017003DE041F61C00C2F2000001900221BF
:1082D000FAF704FD0146019803910321FAF7FEFC29
:1082E00002900398000A8DF8130003988DF811008E
:1082F0000298000A8DF8120002988DF810009DF87F
:1083000011109DF812209DF81300FFF7E3FD20B92E
:10831000FFE700208DF8170012E09DF810000728F5
:1083200004DBFFE701208DF81000FFE741F61C0198
:10833000C2F200010498C86001208DF81700FFE721
:108340009DF8170006B080BD80B584B003900399F6
:108350004878C97840EA0120029003990878897822
:1083600040EA0120019041F61C00C2F20000022107
:10837000FAF7B4FC029988420BD1FFE741F61C00E2
:10838000C2F200000321FAF7A9FC019988420FD03C
:10839000FFE7029A41F61C00C2F2000000900221A1
:1083A000FAF7B4FC0098019A0321FAF7AFFCFFE753
:1083B00041F61C00C2F200000121FAF78FFC43F2E3
:1083C000A52188420AD0FFE741F61C00C2F2000056
:1083D000012143F2A522FAF799FCFFE704B080BD22
:1083E00084B003908DF80B108DF80A2000200190C6
:1083F0000090039800F5FA6001909DF80B000228A8
:108400002DD8FFE79DF80B00172148434CF21D7152
:10841000C1F67141A0FB01109DF80A1008440199B2
:108420000844013900EB910048F21F52C5F2EB12EB
:10843000A1FB0221A0EB511000EBD110043044F657
:108440002511C2F29241A0FB0121421A01EB520216
:108450009108C900A1EB9201401A00902BE09DF811
:108460000B00172148434CF21D71C1F67141A0FB6E
:1084700001109DF80A1008440199084400EB91008E
:1084800048F21F52C5F2EB12A1FB0221A0EB5110E2
:1084900000EBD110023044F62511C2F29241A0FB4C
:1084A0000121421A01EB52029108C900A1EB92018D
:1084B000401A0090FFE79DF8000004B070470000EC
:1084C00080B584B00390029100208DF807000398D6
:1084D000FFF7A0FC20B1FFE701208DF8070013E0B3
:1084E000BDF80A00039909680862BDF808000399FD
:1084F000096848620398FFF7B9FC20B1FFE7012043
:108500008DF80700FFE7FFE79DF8070004B080BD86
:1085100083B002900191ADF80220029818B1FFE7F4
:10852000019808B9FFE723E00198008802990880C4
:108530000198408802994880019880880299888033
:108540000198C0880299C880019800890299088121
:10855000019840890299488101988089029988810F
:1085600002990020C881BDF8020002990882FFE745
:1085700003B0704780B584B00390029100208DF85D
:1085800007000398FFF746FC20B1FFE701208DF8B4
:10859000070013E0BDF80A00039909688861BDF877
:1085A000080003990968C8610398FFF75FFC20B1D0
:1085B000FFE701208DF80700FFE7FFE79DF80700C0
:1085C00004B080BD704700007047000080B596B0D1
:1085D0000CA801902821F7F776FE0198002202925C
:1085E0000B920A92099208920792069205920492BF
:1085F000039209210C914FF480310D910E920122CA
:10860000109212920222139214914FF4E0111591DC
:10861000FAF726F818B1FFE7F8F798FBFFE70F2005
:10862000079002210891002009904FF480620A927D
:108630000B9007A8F9F736FE18B1FFE7F8F786FBAD
:10864000FFE7032003904FF4007004904FF40040C4
:10865000059003A8F9F742FD18B1FFE7F8F776FB9C
:10866000FFE716B080BD00007047000080B541F6FE
:108670008800C2F20000FBF7E9FA80BD80B541F640
:108680008800C2F20000FBF7E1FA80BD80B541F638
:108690008800C2F20000FBF7D9FA80BD80B541F630
:1086A0008800C2F20000FBF7D1FA80BD80B541F22C
:1086B000B860C2F20000FEF75DFF80BD80B541F6F4
:1086C0001810C2F20000FBF7C1FA40F20400C2F237
:1086D0000000007838B1FFE740F20401C2F2000167
:1086E00000200870FFE780BD80B541F2E860C2F26B
:1086F0000000FEF73FFF80BD83B002900191029819
:1087000000680090029842F60041C4F201018842DC
:1087100015D0FFE70298B0F1804F10D0FFE7029824
:1087200040F20041C4F20001884208D0FFE70298FD
:1087300040F60001C4F2000188420AD1FFE7009828
:1087400020F0700000900198416800980843009064
:10875000FFE7029842F60041C4F20101884215D0B9
:10876000FFE70298B0F1804F10D0FFE7029840F287
:108770000041C4F20001884208D0FFE7029840F6A9
:108780000001C4F2000188420AD1FFE7009820F4FA
:10879000407000900198C168009808430090FFE77E
:1087A000009820F0800001994969084300900098E2
:1087B00002990860019880680299C862019800686F
:1087C00002998862029842F60041C4F2010188428F
:1087D00005D1FFE70198006902990863FFE7029954
:1087E0000120486102980069C00730B1FFE7029993
:1087F000086920F001000861FFE703B0704700003E
:1088000085B00490039102920193049880680090CF
:10881000009820F47F40009003980299019A41EA61
:108820000221014300980843009000980499886051
:1088300005B0704783B00290019102988068009063
:10884000009820F07000009001980099084340F0D3
:108850000700009000980299886003B070470000FC
:1088600085B00490039102920498006A00900499E4
:10887000086A20F00100086204988069019001985C
:1088800020F0F00001900299019840EA0110019057
:10889000009820F00A000090039900980843009087
:1088A00001980499886100980499086205B070479E
:1088B00085B00490039102920498006A0090049994
:1088C000086A20F0100008620498806901900198FD
:1088D00020F4704001900299019840EA0130019023
:1088E000009820F0A00000900399009840EA011041
:1088F000009001980499886100980499086205B075
:108900007047000080B582B001900198406A0090E5
:1089100000990020C8850099C8840098FBF77EFC68
:1089200002B080BD84B00390FFE7FFE703980068C2
:1089300050E8030F20F490700290FFE7029903982B
:10894000026842E803100028F0D1FFE7FFE7FFE7E5
:10895000FFE70398006850E8050F20F00100019040
:10896000FFE701990398026842E805100028F0D15A
:10897000FFE7FFE70398006B012814D1FFE7FFE74B
:10898000FFE70398006850E8030F20F01000009004
:10899000FFE700990398026842E803100028F0D12D
:1089A000FFE7FFE7FFE70399202081F842000399E2
:1089B0000020086304B0704780B582B00190019830
:1089C0000168C86820F04000C8600199202081F843
:1089D00041000198FBF7A6FF002002B080BD000017
:1089E00080B586B00490049890F84200222840F0A8
:1089F000A480FFE704988068B0F5805F15D1FFE799
:108A00000498006988B9FFE7002003900498806A01
:108A100002900498006840686FF35F200299088014
:108A20000499886A0230886225E00498806A03907D
:108A30000020029004988068B0F5805F08D0FFE7BE
:108A40000498806850B9FFE70498006930B9FFE7DF
:108A50000498006840680399087007E0049800686B
:108A6000406800F07F0003990870FFE70499886A66
:108A700001308862FFE70499C88D0138C885000479
:108A8000002856D1FFE704980168C86820F020004C
:108A9000C86004980168C86820F48070C8600498B1
:108AA0000168486920F0010048610499202081F89C
:108AB00042000499002048630498006B012830D1DB
:108AC000FFE7049900200863FFE7FFE704980068C8
:108AD00050E8030F20F010000190FFE7019904987F
:108AE000026842E803100028F0D1FFE7FFE704988E
:108AF00000680068C00600280ED5FFE7FFE70020E9
:108B0000009004980068006800900498006840682D
:108B100000900098FFE7FFE70498818DFBF7C2F90A
:108B200003E00498FBF7C0FEFFE700208DF8170074
:108B300007E000208DF8170003E002208DF81700F1
:108B4000FFE79DF8170006B080BD000080B584B037
:108B5000039003980068006920F44050039A11685C
:108B6000D26810430861039988680A69496910430B
:108B70000843029003980068C06841F20C61884382
:108B80000299084303990968C8600398006840691E
:108B900020F44070039A1168926910434861039869
:108BA000006843F60001C4F20101884204D1FFE7E6
:108BB000F9F7E6FC019003E0F9F7D0FC0190FFE73C
:108BC000019819214843039A116852689200B0FB3A
:108BD000F2FC48F21F52C5F2EB12ACFB0230430923
:108BE000642003FB10CC322000EB0C10A0FB02022F
:108BF000F02000EA521000EB0310C2F343121044BD
:108C0000886004B080BD000083B002900191ADF88F
:108C10000220019802998862BDF8020002998885B5
:108C2000BDF802000299C8850299002048640299A3
:108C3000222081F842000298006938B1FFE70298CB
:108C40000168C86840F48070C860FFE70298016856
:108C5000486940F00100486102980168C86840F026
:108C60002000C860002003B07047000083B001906E
:108C7000019890F8410021283AD1FFE701988068D7
:108C8000B0F5805F13D1FFE70198006978B9FFE77D
:108C90000198006A0090009800886FF35F200199A6
:108CA000096848600199086A0230086208E0019A80
:108CB000106A411C11620078019909684860FFE759
:108CC0000199C88C0138C884000468B9FFE701988D
:108CD0000168C86820F08000C86001980168C86811
:108CE00040F04000C860FFE700208DF80B0003E073
:108CF00002208DF80B00FFE79DF80B0003B07047D2
:108D000080B541F2B860C2F20000FEF73FFD80BDC1
:108D100080B541F2E860C2F20000FEF737FD80BD89
:108D2000FFE7FEE781B08DF803009DF903000028FE
:108D30000ED4FFE79DF9031001F01F0201209040BF
:108D40004A094EF20011CEF2000141F82200FFE77D
:108D500001B070474EF60C50CEF200000068C0F330
:108D60000220704782B08DF8070000919DF907003E
:108D700000280AD4FFE7009800019DF907104EF281
:108D80000042CEF2000288540BE0009800019DF8EA
:108D9000071001F00F014EF61452CEF20002885473
:108DA000FFE702B07047000083B00290029800F025
:108DB000070000904EF60C51CEF2000108680190B9
:108DC00001984FF6FF02104001900198009A40EA86
:108DD00002200022C0F2FA5210430190019808606C
:108DE00003B0704780B582B00190009140F210212D
:108DF000C2F20001FF20087040F21121C2F200010E
:108E00000870FFE70098411E009138B3FFE740F279
:108E10001023C2F20003187801994A1C01920978C4
:108E2000414042F26840C2F20000016040F211216C
:108E3000C2F200010A78D0F800E040F2050CC2F25C
:108E4000000C1CF80EC082EA0C021A70026840F294
:108E50000510C2F20000805C0870D3E740F21020D9
:108E6000C2F20000007840F21121C2F2000109783C
:108E700040EA012002B080BD83B002900191002041
:108E80000090FFE700980199884245DAFFE7009BD0
:108E900041F63D20C2F2000050F83310029AC3EBB5
:108EA000C30342F82310009A00EBC2004068029905
:108EB000C2EBC20201EB82014860009A501C029989
:108EC000C2EBC20201EB8201088302980099C1EB58
:108ED000C10100EB81010120888102980099C1EB5A
:108EE000C10100EB81011620887302980099C1EB43
:108EF000C10100EB81011220087502980099C1EBB5
:108F0000C10100EB8101487D40F001004875FFE799
:108F1000009801300090B5E703B0704780B584B089
:108F20000390ADF80A108DF80920ADF80630002046
:108F30000090FFE700989DF80910884212DAFFE7D9
:108F4000BDF80A10012000FA01F20399C8685040E8
:108F5000C860BDF80600F8F781FBFFE70098013014
:108F60000090E7E704B080BD80B590B000200A9083
:108F70000F90F8F7F7FEFFF729FBFDF727FBFDF74A
:108F800069FCFDF731FDFDF751FDFDF7A7FCFDF78D
:108F9000E7FCFDF7C3FAFDF7F5FAFDF7B7FBFDF7C0
:108FA000D9FBFDF72FFC41F20000C4F201000D21B6
:108FB0000A223223FFF7B2FF41F2B860C2F200008A
:108FC0000B9041F6A811C2F2000141F6D002C2F2A4
:108FD0000002FDF72FFA0A9B0B98032141F2883219
:108FE000FDF7E6F90A990B98FDF75AFA41F2E860A5
:108FF000C2F2000041F6F011C2F2000141F6601227
:10900000C2F20002FDF716FA18B1FFE7F7F79EFE6D
:10901000FFE741F2E860C2F2000041F21871C2F2CB
:1090200000018160002141F288320123FDF7C0F97F
:1090300018B1FFE7F7F78AFEFFE7002009908DF8E7
:109040003B0041F68800C2F20000F7F7CBFC00F0CD
:109050009FFA41F25060C2F2000008900068C17AA5
:1090600042F22010C2F20000FFF706FF08980068E5
:10907000C17A40F27830C2F20000A0F86019FEF721
:10908000E9FF09980D90FFE70D98FE280BDCFFE73C
:109090000D9841F2FC41C2F200010854FFE70D981F
:1090A00001300D90F0E7FFE742F22011C2F200011B
:1090B000049101200690087540F27830C2F2000059
:1090C000039041F2F841C2F200010291F7F746FE27
:1090D0000299039841F25062C2F200020592002305
:1090E0000793F7F7CBF900F0B3FA059904980968EC
:1090F000C97AFFF7C1FE05980699079AF7F7C0FDF0
:1091000007980C90FFE70C9841F25061C2F2000101
:109110000968C97A884260DAFFE70C98C0EBC001A1
:1091200041F69020C2F2000010F831008008C0071C
:1091300068B1FFE70C98C0EBC00141F69020C2F285
:10914000000000EBC101488801304880FFE70C981F
:10915000C0EBC00141F69020C2F20000009000EB8D
:10916000C100F7F7CDFC00980C990191C1EBC1014A
:1091700000EBC100006A0021C4F2201100F084FC61
:1091800000F0D2FB019A014640F27830C2F20000B2
:1091900020F8121090F87609C0F3001141F63C2037
:1091A000C2F200000170007848B1FFE740F60C0100
:1091B000C4F20101086840F48060086008E040F6ED
:1091C0000C01C4F20101086820F480600860FFE728
:1091D000FFE70C9801300C9095E765E785B00490A7
:1091E000039100200290FFE702980399884280F2E1
:1091F000CB81FFE700200190FFE7019841F2506129
:10920000C2F200010968C97A884280F2B881FFE79A
:10921000019800900F2800F2AD810099DFE811F06D
:109220001000290043005D0077009100AB00C500ED
:10923000DD00F60010012A0144015E01780192016F
:109240000299019800EB0110C0EBC00241F690209A
:10925000C2F2000010F8320000F00102049800EBA6
:10926000410191F8840900F0FE00104481F884095E
:1092700080E10299019800EB0110C0EBC00241F6B9
:109280009020C2F2000010F8320000F001020498B1
:1092900000EB410191F8840900F0FD0040EA420032
:1092A00081F8840966E10299019800EB0110C0EB96
:1092B000C00241F69020C2F2000010F8320000F027
:1092C0000102049800EB410191F8840900F0FB00D1
:1092D00040EA820081F884094CE10299019800EB90
:1092E0000110C0EBC00241F69020C2F2000010F85D
:1092F000320000F00102049800EB410191F884096A
:1093000000F0F70040EAC20081F8840932E10299D6
:10931000019800EB0110C0EBC00241F69020C2F2B0
:10932000000010F8320000F00102049800EB410147
:1093300091F8840900F0EF0040EA021081F88409F6
:1093400018E10299019800EB0110C0EBC00241F650
:109350009020C2F2000010F8320000F001020498E0
:1093600000EB410191F8840900F0DF0040EA42106F
:1093700081F88409FEE00299019800EB0110C0EB2E
:10938000C00241F69020C2F2000010F8320000F056
:109390000102049800EB410191F8840900F0BF003C
:1093A00040EA821081F88409E4E00299019800EB18
:1093B0000110C0EBC00241F69020C2F2000010F88C
:1093C0003220049800EB410191F8840900F07F00FD
:1093D00040EAC21081F88409CCE00299019800EBC0
:1093E0000110C0EBC00241F69020C2F2000010F85C
:1093F000320000F00102049800EB410191F8850968
:1094000000F0FE00104481F88509B3E0029901984C
:1094100000EB0110C0EBC00241F69020C2F2000048
:1094200010F8320000F00102049800EB410191F8BD
:10943000850900F0FD0040EA420081F8850999E0C5
:109440000299019800EB0110C0EBC00241F6902098
:10945000C2F2000010F8320000F00102049800EBA4
:10946000410191F8850900F0FB0040EA820081F893
:1094700085097FE00299019800EB0110C0EBC00262
:1094800041F69020C2F2000010F8320000F0010214
:10949000049800EB410191F8850900F0F70040EADB
:1094A000C20081F8850965E00299019800EB01107E
:1094B000C0EBC00241F69020C2F2000010F832006A
:1094C00000F00102049800EB410191F8850900F0D9
:1094D000EF0040EA021081F885094BE002990198FB
:1094E00000EB0110C0EBC00241F69020C2F2000078
:1094F00010F8320000F00102049800EB410191F8ED
:10950000850900F0DF0040EA421081F8850931E06A
:109510000299019800EB0110C0EBC00241F69020C7
:10952000C2F2000010F8320000F00102049800EBD3
:10953000410191F8850900F0BF0040EA821081F8EE
:10954000850917E00299019800EB0110C0EBC002F9
:1095500041F69020C2F2000010F83220049800EB8F
:10956000410191F8850900F07F0040EAC21081F8BE
:109570008509FFE7FFE70198013001903DE6FFE72D
:109580000298013002902FE6002005B070470000DD
:1095900080B582B000200190FFE7019841F2506150
:1095A000C2F200010968C97A88424EDAFFE70199E0
:1095B000CB17C1EBC10241F69020C2F2000000EBD4
:1095C000C202936251620199C1EBC10100EBC10279
:1095D00040F63541C0F60001C2F82D100199C1EBEB
:1095E000C10100EBC1021F2182F82C100199C1EBCF
:1095F000C10100EBC1020021C4F2A0119160019BE6
:1096000040F27831C2F2000101F6A612142122F8CC
:1096100013100199C1EBC10100EBC1030121998134
:10962000019B02EB4302A2F8C8100199C1EBC101F2
:1096300000EBC10141F25060C2F20000F7F7ACF953
:10964000FFE7019801300190A7E702B080BD00005C
:1096500080B586B000200590FFE7059841F2506183
:10966000C2F200010968C97A884280F28D80FFE762
:109670000598C0EBC00141F69020C2F2000000EB5B
:10968000C10081680391016A0491808900F068F942
:109690000146039800F0C4FA0146049800F0EFF880
:1096A000B0B9FFE70599012000FA01F340F27831E3
:1096B000C2F20001B1F898291A43A1F89829059A35
:1096C00000FA02F2B1F894099043A1F8940956E027
:1096D0000598C0EBC00141F69020C2F2000000EBFB
:1096E000C10081680191016A0291808900F038F916
:1096F0000146019800F04CF80146029800F0C6F8C7
:10970000B0B9FFE70599012000FA01F340F2783182
:10971000C2F20001B1F898299A43A1F89829059A54
:1097200000FA02F2B1F894091043A1F8940925E077
:109730000598C0EBC00141F69020C2F2000000EB9A
:10974000C1008168006A00F085F8B0B1FFE70599B3
:10975000012000FA01F340F27831C2F20001B1F8C1
:1097600094299A43A1F89429059A00FA02F2B1F8D3
:1097700098099043A1F89809FFE7FFE7FFE7FFE7A3
:1097800005980130059068E7002006B080BD000014
:1097900090EA010F48BF81F0004100F14882421A6F
:1097A0003CBF801A89184FEAD052A2EBD1534FF038
:1097B0007F4C1CEA410F18BF9CEA026F00F03B800F
:1097C0004FF0004C4CEA00204CEA012121FA03FC46
:1097D00010EB0C0C1ED202F1FF325FEA1C2040EBB2
:1097E000C25038BF70471CF07F0F4FEA400C18BFC3
:1097F000BCF17F4F38BF7047C3F12003994008BFC9
:1098000020F00100BCF17F4F38BF7047A0F1C0408D
:1098100000F001BA4FEA3C00000A40EBC25028BFFA
:109820001CF0FF0F4FEA400CE6D018BFBCF17F4F91
:1098300038BF7047EAE79CEA026F05D010EA5C0F78
:1098400008BF00F00040704710B500F09EF900BF5F
:1098500064FBBE3E10B500F033F80CBF01200020C1
:1098600010BD10B500F02CF814BF0120002010BD71
:1098700010B500F0A1F88CBF0120002010BD10B57C
:1098800000F09AF82CBF0120002010BD10B500F0A8
:10989000C7F894BF0120002010BD10B500F0C0F83B
:1098A00034BF0120002010BD401058BFC0F140401F
:1098B000491058BFC1F140418142EFF30080704729
:1098C00050EA010C00F113801CF5000F58BFBCF5E5
:1098D000000F01D48842704707D710F5000F58BF1A
:1098E00011F5000F15D488427047894270471CF566
:1098F000000F04D5BCF5000FF7D5814270474FF03B
:10990000807C1CEB400F38BF1CEB410F01D2814221
:10991000704710B500F039F9922449004FF000501B
:109920004FF08051FFF7C0BF41000B0ED3F19E02F4
:1099300008D950F400034FEA032323FA02F048BF8A
:109940004042704710B500F020F900BF49922480D2
:10995000002070476FF0004282EA2000704700004C
:1099600010F0004148BF4042B0FA80F310FA03F211
:10997000C3F19D030BD051EAC35101EB12205306F2
:1099800038BF704700F1010008BF20F001007047A8
:10999000B0FA80F310FA03F2C3F19D030AD0D9059F
:1099A00001EB1220530638BF704700F1010008BFD9
:1099B00020F001007047000050EA010C00F1138014
:1099C0001CF5000F58BFBCF5000F01D4884270474A
:1099D00007D710F5000F58BF11F5000F15D48842B6
:1099E0007047894270471CF5000F04D5BCF5000F85
:1099F000F7D5814270474FF0807C1CEB400F38BF99
:109A00001CEB410F01D28142704710B500F0BDF848
:109A1000922449004FF080504FF00051FFF744BFAF
:109A200050EA010C00F113801CF5000F58BFBCF583
:109A3000000F01D48842704707D710F5000F58BFB8
:109A400011F5000F15D488427047894270471CF504
:109A5000000F04D5BCF5000FF7D5814270474FF0D9
:109A6000807C1CEB400F38BF1CEB410F01D28142C0
:109A7000704710B500F089F8922449004FF000506B
:109A80004FF08051FFF710BF4FF47F0C1CEAD0124B
:109A90001EBF1CEAD11392EA0C0F93EA0C0F00F0E0
:109AA000478090EA010F48BF42F480724FF0004CAB
:109AB0004CEA00204CEA012102EB0302A0FB011357
:109AC000A2F50002002918BF43F001035B0028BF84
:109AD0004FEA330342EB22425FEA132C4CEBC250B5
:109AE0002EBFBCEB436FB2F57C0F70474FEA036C9F
:109AF000BCF1004F08BF20F00100B2F57C0F38BF69
:109B000070470BD582F0FF0212F5803FC8BF704747
:109B100000F1C040D8BF00F00040704700F5000CD5
:109B20005FEA4C0C48BF7047B0F1C04000F073B81A
:109B30000CEAD11390EA010F48BF42F480726245EB
:109B400038BF634504D280EA010000F0004070474E
:109B500010B500F01AF800BF8900013E00F007B808
:109B600000F009B85FEA410C5FEA1C6C08D080EA9B
:109B7000010000F050B85FEA400C5FEA1C6CF6D1BF
:109B80004FF00040A0F5800070470EF1020E2EF05D
:109B9000030E5EF8044B244204D44FEA4102B2F1B2
:109BA0007F4F11D84FEA4003B3F17F4F0CD80ED14D
:109BB0004FEAD07C0CEB4C0C0CF1020CB2F17F4F55
:109BC00008BF4CEBD17C04E04FF0080C01E04FEAF9
:109BD000D17C0CEB4C0324FA03F404F00704B4F139
:109BE000040C06D20EEB840CBDE810404CF0010CC6
:109BF0006047DFE80CF0070802024FF00040A0F5D4
:109C0000800010BD0846420018BFD2F1807288BFA4
:109C100000F0004010BDFF2141EAD050C005704760
:109C200090EA010F48BF81F000413FF5B8AD421AFC
:109C300004D882F00042A0EB020011444FEAD05257
:109C4000A2EBD1534FF07F4C1CEA410F18BF9CEAA6
:109C5000026F4AD04FF0004C4CEA00204CEA012140
:109C600021FA03FCB0EB0C0C0FD412F0FE0F36D02F
:109C70005FEA4C001DD5001240EBC25038BF704760
:109C80001CF03F0F18BF70470BE05FEA1C20A2F1E9
:109C9000010240EBC25038BF70471CF07F0F18BF65
:109CA0007047C3F12003994014BF401E20F001000B
:109CB00070474FEA1223800808BF7047B0FA80FC53
:109CC000A2EB0C02CCF1280C60FA0CF093EA122FF4
:109CD00004BF00EBC25070474FEAC3707047130ACD
:109CE0005FEADC1008BF7047F6E79CEA026F04D019
:109CF00010EA5C0F08BF0020704710B5FFF745FF62
:109D000040DFF63E81F00040704700000000000098
:109D10000000010203040607080900000000010218
:109D2000030402030405060708090A0B0C0D0E0FB5
:109D30001010010202030405060708090A0B0C0DA6
:109D40000E0F101001021F1C1F1E1F1E1F1F1E1FA3
:109D50001E1F4E494F2D313200000000809D00082B
:109D6000000000201802000050010008C09E0008FA
:109D70001802002058280000B80100080000000068
:109D8000200E00127A000100C1814001C080410410
:109D9000610C2108E118A11C011A300116380136A6
:109DA00060012E70012F6000FF00C0C101C30302DB
:109DB000C2C60607C705C5C404CC0C0DCD0FCFCE57
:109DC0000E0ACACB0BC90908C8D81819D91BDBDA87
:109DD0001A1EDEDF1FDD1D1CDC14D4D515D71716A7
:109DE000D6D21213D311D1D010F03031F133F3F2B7
:109DF0003236F6F737F53534F43CFCFD3DFF3F3E97
:109E0000FEFA3A3BFB39F9F83828E8E929EB2B2A26
:109E1000EAEE2E2FEF2DEDEC2CE42425E527E7E6E6
:109E20002622E2E323E12120E0A06061A163A3A256
:109E30006266A6A767A56564A46CACAD6DAF6F6ED6
:109E4000AEAA6A6BAB69A9A86878B8B979BB7B7A06
:109E5000BABE7E7FBF7DBDBC7CB47475B577B7B626
:109E60007672B2B373B17170B050909151935352F6
:109E70009296565797559594549C5C5D9D5F9F9E16
:109E80005E5A9A9B5B99595898884849894B8B8AA6
:109E90004A4E8E8F4F8D4D4C8C4484854587474666
:109EA00086824243834181801006400000001C04EA
:109EB000124804000900FFFF01001000000000002C
:04000005080000ED02
:00000001FF
